:020000020000FC
:100000000C946F31189518951895189518951895A2
:100010001895189518951895189518951895189578
:100020001895189518951895189518951895189568
:100030001895189518951895189518951895189558
:100040001895189518951895189518951895189548
:100050000C94770B18951895189518951895189570
:100060001895189518951895189518951895189528
:100070001895189518951895189518951895189518
:100080001895189518951895189518951895189508
:1000900018951895189518951895189518951895F8
:1000A00018951895189518951895189518951895E8
:1000B00018951895189518951895189518951895D8
:1000C00018951895189518951895189518951895C8
:1000D00018951895189518951895189518951895B8
:1000E00018951895189518951895189518951895A8
:1000F0001895189518951895189518951895189598
:100100001895189518951895189518951895189587
:100110001895189518951895189518950C94660BC0
:100120001895189518951895189518951895189567
:10013000189518950C94E80A18951895189518951F
:100140001895189518951895189518951895189547
:100150001895189518951895189518951895189537
:100160001895189518951895189518951895189527
:100170001895189518951895189518951895189517
:100180001895189518951895189518951895189507
:1001900018951895189518951895189518951895F7
:1001A00018951895189518951895189518951895E7
:1001B00018951895189518951895189518951895D7
:1001C00018951895189518951895189518951895C7
:1001D00018951895189518951895189518951895B7
:1001E00018951895189518951895189518951895A7
:1001F00018951895189518951895189544241FBCAE
:1002000037CB7ABC26B8A2BD41F61CBE6EBA0DBE75
:10021000FC0C633C5C1D633E6EE3A33E5C1D633ED1
:10022000FC0C633C6EBA0DBE41F61CBE26B8A2BDE6
:1002300037CB7ABC44241FBC631349BEDBD713BE43
:100240003B43DA3BD34F453EE0C1903ED34F453E62
:100250003B43DA3BDBD713BE631349BE14BEA1BDDB
:100260006FEDFCBDDC252FBEE9383F3FDC252FBEFE
:100270006FEDFCBD14BEA1BD90F90F3F90F90FBF0B
:100280000000803FFE98FFBDE5FF3CBE6A8B31BE9B
:10029000D6704CBC0186593E0595A33E0186593E59
:1002A000D6704CBC6A8B31BEE5FF3CBE1F1F1F00E1
:1002B000000000001C1E1F1F1F1F1F1F1F1F1F1FCE
:1002C0001F1F1E1C00000000001F1F1F1F1F1F1FDD
:1002D0001F1F0F07070F1F1F1F1F1F1F00000000FA
:1002E000001F1F1F1F1F1F00001F1F1F05000104ED
:1002F00003022020052020FF000701040306000759
:10030000010603020506FF2020FF05070006030281
:100310000507000403020000012020FF0507010477
:100320000302050701030302050707042020050750
:1003300007040303050701042020001F2C3D630070
:100340000102040810204000000000010101012406
:10035000212A21302136213A213D214121452149BF
:10036000214D21522157215C212A2A2A2A2A2A2A70
:100370002A2A00003328100032220524C024082530
:100380003A257F25AF25F42539267F26BA26EA2689
:100390002D277D27BB27F7270000B32C10000E293F
:1003A000B32C5C2AB32C772AC12AC52BE72BFF2B51
:1003B000B32CED302B2C442C5C2CB32C742C000073
:1003C000D62E1000C92C082D1B2D302D4F2D7A2D27
:1003D000A52DBF2DD42D472E582E7F2E902EA12E29
:1003E000B22EC92E0000E6301000EC2E302F432F25
:1003F000582F712F9C2FC52FDF2FF42F59306A30C3
:100400008F30A030B130C230D93000013C3739379D
:10041000452C37022C371196360B5B3601B436016A
:100420002C37012C37012C3702B4360548360189A8
:1004300036019636036436029636039236FB00E3A5
:1004400030D000E815E237D100E815E234D100E8F9
:1004500015E231D100E325D000E815E22CD100E30C
:1004600020D000EC13E027D102E01BD000EC13E019
:1004700022D108E016D000EC13E01DD101E011D02C
:1004800000E815E218D100E815E215D106E009D020
:1004900000EC13E010D10CE004D000EC13E00BD121
:1004A00008958A93802FE4E4F6E000810F7B0083B7
:1004B00000E310E000D100916406007F0093640621
:1004C000082F02950F7010916406102B109364068C
:1004D000E4E4F6E000810068008300E310E0EBD084
:1004E000E4E4F6E000810F77008300EF10E0E3D052
:1004F00000916406007F009364068F70009164068B
:10050000082B00936406E4E4F6E0008100680083B1
:1005100000E310E0D0D0E4E4F6E000810F77008340
:1005200000EF10E0C8D0899108958A93802FE4E409
:10053000F6E000810064008300E310E0BCD000918D
:100540006406007F00936406082F02950F701091D7
:100550006406102B10936406E4E4F6E00081006862
:10056000008300E310E0A7D0E4E4F6E000810F7719
:10057000008300EF10E09FD000916406007F00939D
:1005800064068F7000916406082B00936406E4E40F
:10059000F6E000810068008300E310E08CD0E4E422
:1005A000F6E000810F77008300EF10E084D089919E
:1005B00008950E94F434C801A0E007C0B0E0FC0137
:1005C000EA0FFB1F0081B1DFA395B0E0FC01EA0F49
:1005D000FB1F0081002311F0A13180F3E4E00C94B3
:1005E00005355FDF0EE915E2E4DF08951BEC10939B
:1005F000520018E010935000E1E5F0E0108113FF85
:10060000FBCF003221F402EC0093550003C003EC51
:1006100000935500E0E5F0E0008100610083E1E532
:10062000F0E0008104FFFBCF08ED04BF04E000937D
:100630004000E0E5F0E000810E7F0083089504E4CF
:1006400014E000930C0210930D0200E100930102EC
:1006500002E20093020203E00093040203E000932D
:10066000200208E200932102E0E0F2E00081016054
:100670000083089501E00093280200E3009329021B
:10068000089501E00093300208E3009331020895D9
:100690000DE00093200300E40093210300E00093A9
:1006A000220300E50093240300E70093280300EEF3
:1006B00000932A0308950150104098018901232BCB
:1006C000D1F708958A93802F04C008EE1DEF0E9491
:1006D0001C118A95082F802F0023B9F7899108955E
:1006E0000E94F33480E090E0A0E0B0E04EE0442EC1
:1006F0001BC0442D50E0440F551F440F551FFA01F5
:10070000E655FA4D0080118022803380442D50E060
:10071000440F551F440F551FFA01E255FA4D008250
:100720001182228233824A9441E0441610F7EEEAA5
:10073000F5E20083118322833383442423C0042DF4
:1007400010E0000F111F000F111FF801E450FE4FC1
:100750004591559165917491042D10E0000F111F82
:10076000000F111FF801E255FA4D0081118122811D
:1007700033810E947833AC01BD010E941733C80158
:10078000D90143940FE04016D0F28C019D01E5E0C1
:100790000C9404350E94F33480E090E0A0E0B0E0D7
:1007A0004EE0442E1BC0442D50E0440F551F440F13
:1007B000551FFA01EA51FA4D0080118022803380E2
:1007C000442D50E0440F551F440F551FFA01E651C8
:1007D000FA4D00821182228233824A9441E044160B
:1007E00010F7EAEEF5E20083118322833383442479
:1007F00023C0042D10E0000F111F000F111FF8017E
:10080000E450FE4F4591559165917491042D10E08F
:10081000000F111F000F111FF801E651FA4D008162
:100820001181228133810E947833AC01BD010E9485
:100830001733C801D90143940FE04016D0F28C0160
:100840009D01E5E00C9404350E94F33480E090E0D3
:10085000A0E0B0E04EE0442E1BC0442D50E0440F19
:10086000551F440F551FFA01EE5DF94D00801180B0
:1008700022803380442D50E0440F551F440F551FF4
:10088000FA01EA5DF94D00821182228233824A9494
:1008900041E0441610F7E6E2F6E20083118322837A
:1008A0003383442423C0042D10E0000F111F000FD8
:1008B000111FF801E450FE4F4591559165917491D7
:1008C000042D10E0000F111F000F111FF801EA5D49
:1008D000F94D00811181228133810E947833AC016E
:1008E000BD010E941733C801D90143940FE040169F
:1008F000D0F28C019D01E5E00C9404350E94F334A4
:1009000080E090E0A0E0B0E048E0442E1BC0442D21
:1009100050E0440F551F440F551FFA01E25AF94D9C
:100920000080118022803380442D50E0440F551FF9
:10093000440F551FFA01EE59F94D008211822282AF
:1009400033824A9441E0441610F7E2E6F6E200836F
:10095000118322833383442423C0042D10E0000F2D
:10096000111F000F111FF801E85CFD4F45915591D3
:1009700065917491042D10E0000F111F000F111FDD
:10098000F801EE59F94D00811181228133810E94D5
:100990007833AC01BD010E941733C801D9014394DB
:1009A00009E04016D0F28C019D01E5E00C9404357D
:1009B0000E94F33480E090E0A0E0B0E048E0442EF4
:1009C0001BC0442D50E0440F551F440F551FFA0122
:1009D000EE57F94D0080118022803380442D50E085
:1009E000440F551F440F551FFA01EA57F94D008275
:1009F0001182228233824A9441E0441610F7E6E8DD
:100A0000F6E20083118322833383442423C0042D20
:100A100010E0000F111F000F111FF801E85CFD4FDF
:100A20004591559165917491042D10E0000F111FAF
:100A3000000F111FF801EA57F94D00811181228141
:100A400033810E947833AC01BD010E941733C80185
:100A5000D901439409E04016D0F28C019D01E5E0F4
:100A60000C9404350E94F33480E090E0A0E0B0E004
:100A700048E0442E1BC0442D50E0440F551F440F46
:100A8000551FFA01EA55F94D00801180228033800C
:100A9000442D50E0440F551F440F551FFA01E655F1
:100AA000F94D00821182228233824A9441E0441639
:100AB00010F7EAEAF6E200831183228333834424A9
:100AC00023C0042D10E0000F111F000F111FF801AB
:100AD000E85CFD4F4591559165917491042D10E0AE
:100AE000000F111F000F111FF801E655F94D00818D
:100AF0001181228133810E947833AC01BD010E94B3
:100B00001733C801D901439409E04016D0F28C0193
:100B10009D01E5E00C9404350E94F33480E090E000
:100B2000A0E0B0E046E0442E1BC0442D50E0440F4E
:100B3000551F440F551FFA01E653F94D00801180EF
:100B400022803380442D50E0440F551F440F551F21
:100B5000FA01E253F94D00821182228233824A94D3
:100B600041E0441610F7EEECF6E200831183228395
:100B70003383442423C0042D10E0000F111F000F05
:100B8000111FF801E45AFD4F4591559165917491FB
:100B9000042D10E0000F111F000F111FF801E25388
:100BA000F94D00811181228133810E947833AC019B
:100BB000BD010E941733C801D901439407E04016D4
:100BC000D0F28C019D01E5E00C9404350E94F334D1
:100BD00080E090E0A0E0B0E046E0442E1BC0442D51
:100BE00050E0440F551F440F551FFA01EA51F94DCB
:100BF0000080118022803380442D50E0440F551F27
:100C0000440F551FFA01E651F94D008211822282EC
:100C100033824A9441E0441610F7EAEEF6E200838C
:100C2000118322833383442423C0042D10E0000F5A
:100C3000111F000F111FF801E45AFD4F4591559106
:100C400065917491042D10E0000F111F000F111F0A
:100C5000F801E651F94D00811181228133810E9412
:100C60007833AC01BD010E941733C801D901439408
:100C700007E04016D0F28C019D01E5E00C940435AC
:100C80000E94F33480E090E0A0E0B0E046E0442E23
:100C90001BC0442D50E0440F551F440F551FFA014F
:100CA000EE5FF84D0080118022803380442D50E0AB
:100CB000440F551F440F551FFA01EA5FF84D00829B
:100CC0001182228233824A9441E0441610F7E6E012
:100CD000F7E20083118322833383442423C0042D4D
:100CE00010E0000F111F000F111FF801E45AFD4F13
:100CF0004591559165917491042D10E0000F111FDD
:100D0000000F111FF801EA5FF84D00811181228167
:100D100033810E947833AC01BD010E941733C801B2
:100D2000D901439407E04016D0F28C019D01E5E023
:100D30000C9404350E94F03481E035C0482F50E017
:100D4000440F551F440F551FFA01EA5DF84D00800E
:100D5000118022803380482F50E0440F551F440FEC
:100D6000551FFA01E65DF84D00821182228233821E
:100D7000482F50E0440F551F440F551FFA01E25E03
:100D8000F84D0080118022803380482F50E0440FBE
:100D9000551F440F551FFA01EE5DF84D0082118278
:100DA000228233828A95813048F6EAE2F7E20083B4
:100DB000118322833383EAE2F7E240815181628129
:100DC0007381E8E7F2E005911591259134910E9435
:100DD0007833E2E2F7E2008311832283338381E0F8
:100DE0004FC0082F10E0000F111F000F111FF80156
:100DF000E858FD4F4591559165917491082F10E089
:100E0000000F111F000F111FF801E65DF84D008162
:100E10001181228133810E94783328013901082F02
:100E200010E0000F111F000F111FF801E058FD4FD7
:100E30004591559165917491082F10E0000F111F95
:100E4000000F111FF801EE5DF84D00811181228124
:100E500033810E947833A801B901820193010E9475
:100E60005B33E2E2F7E240815181628173810E944B
:100E70001733E2E2F7E20083118322833383839501
:100E8000823008F4AECFE2E2F7E2008111812281E4
:100E90003381E8E00C9401350E94F03481E035C0E4
:100EA000482F50E0440F551F440F551FFA01EA5CCC
:100EB000F84D0080118022803380482F50E0440F8D
:100EC000551F440F551FFA01E65CF84D0082118250
:100ED00022823382482F50E0440F551F440F551F84
:100EE000FA01E25DF84D0080118022803380482FA6
:100EF00050E0440F551F440F551FFA01EE5CF84DAA
:100F000000821182228233828A95813048F6EAE398
:100F1000F7E20083118322833383EAE3F7E240811F
:100F2000518162817381E8E7F2E005911591259185
:100F300034910E947833E2E3F7E200831183228345
:100F4000338381E04FC0082F10E0000F111F000F06
:100F5000111FF801E858FD4F459155916591749125
:100F6000082F10E0000F111F000F111FF801E65CA1
:100F7000F84D00811181228133810E94783328014C
:100F80003901082F10E0000F111F000F111FF80189
:100F9000E058FD4F4591559165917491082F10E0EF
:100FA000000F111F000F111FF801EE5CF84D0081BA
:100FB0001181228133810E947833A801B901820115
:100FC00093010E945B33E2E3F7E240815181628149
:100FD00073810E941733E2E3F7E2008311832283D7
:100FE00033838395823008F4AECFE2E3F7E20081E9
:100FF000118122813381E8E00C9401350E94F034A4
:1010000081E035C0482F50E0440F551F440F551F55
:10101000FA01EA5BF84D0080118022803380482F6E
:1010200050E0440F551F440F551FFA01E65BF84D81
:101030000082118222823382482F50E0440F551FD4
:10104000440F551FFA01E25CF84D008011802280A8
:101050003380482F50E0440F551F440F551FFA01AD
:10106000EE5BF84D00821182228233828A958130B4
:1010700048F6EAE4F7E20083118322833383EAE44B
:10108000F7E24081518162817381E8E7F2E00591E6
:101090001591259134910E947833E2E4F7E20083C0
:1010A00011832283338381E04FC0082F10E0000FAB
:1010B000111F000F111FF801E858FD4F4591559180
:1010C00065917491082F10E0000F111F000F111F80
:1010D000F801E65BF84D00811181228133810E9485
:1010E000783328013901082F10E0000F111F000F7D
:1010F000111FF801E058FD4F45915591659174918C
:10110000082F10E0000F111F000F111FF801EE5BF8
:10111000F84D00811181228133810E947833A8012A
:10112000B901820193010E945B33E2E4F7E240815E
:101130005181628173810E941733E2E4F7E20083F8
:101140001183228333838395823008F4AECFE2E4A7
:10115000F7E20081118122813381E8E00C940135AE
:101160000E94F034842FA52F0E94B832482F50E0FF
:10117000440F551F440F551FFA01EE5AF84D408198
:101180005181628173810E945B33280139010A2FEA
:1011900010E020E030E00E94C332A801B9018201D2
:1011A00093010E94F133482F50E0440F551F440F24
:1011B000551FFA01EE5AF84D4081518162817381C9
:1011C0000E94173390E0880F991F880F991FFC0128
:1011D000EE5AF84D0083118322833383E8E00C94A8
:1011E00001350E94F33480E090E0A0E0B0E048E0F8
:1011F000442E1BC0442D50E0440F551F440F551F73
:10120000FA01E257F84D0080118022803380442D8E
:1012100050E0440F551F440F551FFA01EE56F84D8C
:1012200000821182228233824A9441E0441610F7F0
:10123000E2E9F7E20083118322833383442423C04D
:10124000042D10E0000F111F000F111FF801E857C7
:10125000FD4F4591559165917491042D10E0000F5B
:10126000111F000F111FF801EE56F84D008111817A
:10127000228133810E947833AC01BD010E94173373
:10128000C801D901439409E04016D0F28C019D01B8
:10129000E5E00C9404350E94F33480E090E0A0E097
:1012A000B0E048E0442E1BC0442D50E0440F551FD1
:1012B000440F551FFA01EE54F84D00801180228032
:1012C0003380442D50E0440F551F440F551FFA0141
:1012D000EA54F84D00821182228233824A9441E01E
:1012E000441610F7E6EBF7E2008311832283338381
:1012F000442423C0042D10E0000F111F000F111F04
:10130000F801E857FD4F4591559165917491042D71
:1013100010E0000F111F000F111FF801EA54F84DE3
:1013200000811181228133810E947833AC01BD019B
:101330000E941733C801D901439409E04016D0F246
:101340008C019D01E5E00C9404350E94F33480E0AB
:1013500090E0A0E0B0E048E0442E1BC0442D50E0F7
:10136000440F551F440F551FFA01EA52F84D0080F3
:10137000118022803380442D50E0440F551F440FCC
:10138000551FFA01E652F84D008211822282338203
:101390004A9441E0441610F7EAEDF7E20083118326
:1013A00022833383442423C0042D10E0000F111F37
:1013B000000F111FF801E857FD4F459155916591B8
:1013C0007491042D10E0000F111F000F111FF80180
:1013D000E652F84D00811181228133810E947833D9
:1013E000AC01BD010E941733C801D901439409E043
:1013F0004016D0F28C019D01E5E00C94043510916B
:10140000480001E0009348002091A0003091A20024
:101410000091A2000C7F04600093A2004FB7789463
:10142000E8E4F0E00081016000835091CD01EF938A
:10143000FF930F932F93EBECF1E008ED21E004BF55
:1014400020832F910F91FF91EF9103E00093CD0145
:101450008895109348002093A0003093A2005093E9
:10146000CD014FBF0895EFECF1E0008107FDFBCF08
:101470000895F9DFEFECF1E0008101FF11C006E310
:101480000093CA01EF93FF930F932F93EBECF1E0DE
:1014900008ED21E004BF20832F910F91FF91EF9180
:1014A00008959A938A93C801DEDFFC01E05CF14065
:1014B000F09750F44091A72950E009E010E00E9415
:1014C000BD31800F911F17C0803C01E0900798F458
:1014D0004091A62950E00BE110E00E94BD31980137
:1014E0004091A72950E001E510E00E94BD31200F96
:1014F000311F820F931F082F0093C001892F8F7116
:101500008093C10100E00093C20106E00093CA018C
:10151000EF93FF930F932F93EBECF1E008ED21E0B5
:1015200004BF20832F910F91FF91EF910091C4018F
:101530008991999108950E94F534C801A22F00E085
:101540000093060900E000934608FC01E05CF140CE
:10155000F09750F44091A72950E009E010E00E9474
:10156000BD31800F911F17C0803C01E0900798F4B7
:101570004091A62950E00BE110E00E94BD31980196
:101580004091A72950E001E510E00E94BD31200FF5
:10159000311F820F931F6DDF03E30093CA01082FF1
:1015A0000093C001892F8F718093C10100E00093E7
:1015B000C201A093C40105E30093CA0120DF03E048
:1015C0000093060901E000934608E3E00C94063519
:1015D0009A938A93FA93EA930A927A936A935A9324
:1015E0004A933A932A931A930A930FB6E0E0F2E0F3
:1015F00000810460008300917129039507700093B6
:1016000071290091712910E0000F111FF801E25FAC
:10161000F74D0081118100933A0310933B03009131
:10162000712910E0000F111FF801E250F84D008100
:10163000118100933803109339030091742900231A
:10164000B1F10091BE281091BF28212F220F220B4B
:10165000322F4091712950E0440F551F440F551F00
:10166000FA01E258F74D4081518162817381400F48
:10167000511F621F731F4083518362837383809164
:10168000D2289091D32801968093D2289093D32882
:101690000091D4281091D5288017910741F400E0DB
:1016A0000093742910E00093D2281093D3280FBE22
:1016B000099119912991399149915991699179919A
:1016C0000990E991F9918991999118952A931A9322
:1016D0000A932FB700911002109111020093BE28B7
:1016E0001093BF282FBF09911991299118955A92EB
:1016F0004A92BA93AA939A938A93FA93EA933A9264
:101700002A921A920A927A936A935A934A933A9334
:101710002A931A930A935FB600917429002309F063
:1017200075C500919829002309F100919829102F7F
:101730001A9510939829002339F400E00093982912
:1017400000E00093400912C000918C291091992962
:10175000019F4091982950E080010E94BD3143E0F3
:101760000E94D13100936A0910936B09009182297C
:101770000E5F0093902980E037C050919029482F48
:10178000642F082F10E0000F111F000F111FF80128
:10179000E258F74D008111812281338142E00E949D
:1017A0002B32462FDDDC0E94C532482F50E0440F1B
:1017B000551F440F551FFA01E256F74D0083118360
:1017C0002283338300E010E020E030E0482F50E037
:1017D000440F551F440F551FFA01E258F74D00837F
:1017E0001183228333838395883038F20FEF00937F
:1017F000742900E010E020E030E0E6EEF8E200833B
:10180000118322833383E2EEF8E200831183228383
:101810003383EEEDF8E2008311832283338300E00B
:1018200010E020E030E0E2EAF9E200831183228355
:1018300033834424C9C0042D10E0000F111F000F92
:10184000111FF801E256F74D408151816281738189
:10185000042D10E0000F111F000F111FF801E256B8
:10186000F74D00811181228133810E9403320E9451
:10187000B832E2EAF9E240815181628173810E94CB
:101880001733E2EAF9E20083118322833383EEED1A
:10189000F8E200811181228133810E94B832C801AF
:1018A000D901042D10E0000F111F000F111FF801C6
:1018B000E256F74D00811181228133810E94B832B6
:1018C000442D50E0440F551F440F551FFA01E25EAE
:1018D000F74D40815181628173810E947833AC0160
:1018E000BD010E9417330E94C532EEEDF8E200837D
:1018F000118322833383E2EEF8E200811181228199
:1019000033810E94B832C801D901042D10E0000FC4
:10191000111F000F111FF801E256F74D00811181D0
:10192000228133810E94B832442D50E0440F551F6C
:10193000440F551FFA01E25CF74D408151816281ED
:1019400073810E947833AC01BD010E9417330E945D
:10195000C532E2EEF8E20083118322833383E6EEA0
:10196000F8E200811181228133810E94B832C801DE
:10197000D901042D10E0000F111F000F111FF801F5
:10198000E256F74D00811181228133810E94B832E5
:10199000442D50E0440F551F440F551FFA01E25AE1
:1019A000F74D40815181628173810E947833AC018F
:1019B000BD010E9417330E94C532E6EEF8E20083B3
:1019C000118322833383439408E0401608F433CF15
:1019D00040E050E060E071E4E2EAF9E20081118168
:1019E000228133810E94F1330E945C39E2EAF9E2FC
:1019F000008311832283338300919429013099F469
:101A0000E2EAF9E200811181228133810E94C5322C
:101A10004091D8285091D9280E94D7310093D028DE
:101A20001093D12814C0E2EAF9E2008111812281E9
:101A300033810E94C5324091D8285091D928440F53
:101A4000551F0E94D7310093D0281093D1280091C0
:101A5000912910E0F801E15CFC4F449150E00091C5
:101A6000D0281091D1280E94D7310093D02810930C
:101A7000D12800919529023051F40091D02810917D
:101A8000D128169507950093D0281093D128EEED14
:101A9000F8E20081118122813381E2EFF8E20083D4
:101AA000118322833383E2EEF8E2008111812281E7
:101AB0003381E6EFF8E20083118322833383E6EE7D
:101AC000F8E20081118122813381EEEFF8E2008398
:101AD000118322833383EAE0F9E2008111812281BC
:101AE0003381EEEFF8E24081518162817381041706
:101AF0001507260737077CF4EAE0F9E20081118137
:101B0000228133810F5F1F4F2F4F3F4F008311837F
:101B1000228333830EC0EAE0F9E200811181228141
:101B200033810150104020403040008311832283D4
:101B30003383E6E0F9E20081118122813381E2EF13
:101B4000F8E24081518162817381041715072607ED
:101B500037077CF4E6E0F9E20081118122813381CC
:101B60000F5F1F4F2F4F3F4F00831183228333831B
:101B70000EC0E6E0F9E2008111812281338101503B
:101B80001040204030400083118322833383E2E001
:101B9000F9E20081118122813381E6EFF8E2408190
:101BA00051816281738104171507260737077CF47A
:101BB000E2E0F9E200811181228133810F5F1F4F42
:101BC0002F4F3F4F00831183228333830EC0E2E007
:101BD000F9E20081118122813381015010402040BF
:101BE00030400083118322833383009173290023C3
:101BF00039F100E000937329E2EFF8E200811181EE
:101C000022813381E6E0F9E200831183228333836A
:101C1000E6EFF8E20081118122813381E2E0F9E20E
:101C20000083118322833383EEEFF8E20081118178
:101C300022813381EAE0F9E2008311832283338336
:101C4000E6E0F9E20081118122813381E2EFF8E2DE
:101C50004081518162817381401B510B620B730B78
:101C60004083518362837383E2E0F9E20081118152
:101C700022813381E6EFF8E24081518162817381F4
:101C8000401B510B620B730B408351836283738340
:101C9000EAE0F9E20081118122813381EEEFF8E27E
:101CA0004081518162817381401B510B620B730B28
:101CB00040835183628373830091DC281091DD2877
:101CC000013020E0120709F020C100919429023070
:101CD00009F4E7C000918E290130B9F5E2EFF8E28E
:101CE00000811181228133810E94B8320E947003E9
:101CF0000E94C532EAE2F9E2008311832283338332
:101D0000E6EFF8E200811181228133810E94B8322E
:101D10000E94CA030E94C532EEE2F9E200831183F9
:101D200022833383EEEFF8E2008111812281338137
:101D30000E94B8320E9424040E94C532E6E2F9E211
:101D4000008311832283338304C100918E290230E2
:101D5000B9F5E2EFF8E200811181228133810E941E
:101D6000B8320E947E040E94C532EAE2F9E20083A2
:101D7000118322833383E6EFF8E20081118122810F
:101D800033810E94B8320E94D8040E94C532EEE22C
:101D9000F9E20083118322833383EEEFF8E20081BE
:101DA0001181228133810E94B8320E9432050E9443
:101DB000C532E6E2F9E20083118322833383C9C08E
:101DC00000918E290330B9F5E2EFF8E2008111812C
:101DD000228133810E94B8320E948C050E94C53254
:101DE000EAE2F9E20083118322833383E6EFF8E22B
:101DF00000811181228133810E94B8320E94E60560
:101E00000E94C532EEE2F9E200831183228333831C
:101E1000EEEFF8E200811181228133810E94B83215
:101E20000E9440060E94C532E6E2F9E20083118377
:101E3000228333838EC0E2EFF8E200811181228198
:101E400033810E94B8320E949A060E94C532EAE2AB
:101E5000F9E20083118322833383E6EFF8E2008105
:101E60001181228133810E94B8320E944C070E9466
:101E7000C532EEE2F9E20083118322833383EEEF71
:101E8000F8E200811181228133810E94B832B6D8F4
:101E90000E94C532E6E2F9E2008311832283338394
:101EA00058C0E2EFF8E200811181228133810E9463
:101EB000B83297D90E94C532EAE2F9E20083118371
:101EC00022833383E6EFF8E200811181228133819E
:101ED0000E94B832E0D90E94C532EEE2F9E20083F6
:101EE000118322833383EEEFF8E200811181228196
:101EF00033810E94B83229DA0E94C532E6E2F9E263
:101F0000008311832283338324C0E2EFF8E200814F
:101F1000118122813381EAE2F9E200831183228375
:101F20003383E6EFF8E20081118122813381EEE212
:101F3000F9E20083118322833383EEEFF8E200811C
:101F4000118122813381E6E2F9E200831183228349
:101F5000338300918929009500938929009189296B
:101F6000002309F023C1EAE2F9E200811181228114
:101F70003381E6E3F9E24081518162817381040F8C
:101F8000151F261F371FE2E4F9E200831183228325
:101F90003383EEE2F9E20081118122813381EAE3A9
:101FA000F9E24081518162817381040F151F261F60
:101FB000371FE6E4F9E20083118322833383E6E2EC
:101FC000F9E20081118122813381E2E3F9E240816B
:101FD000518162817381040F151F261F371FEEE3A5
:101FE000F9E20083118322833383EEEFF8E200816C
:101FF000118122813381EAE5F9E2408151816281D8
:102000007381040F151F261F371FEEE5F9E20083C9
:1020100011832283338300918A29009500938A29B2
:1020200000918A29002309F090C0E2E4F9E20081DE
:10203000118122813381EAE4F9E240815181628198
:102040007381040F151F261F371F43E050E0609176
:10205000952970E0461B570B652F660F660B762F90
:102060000E945632EAEEF8E2008311832283338322
:10207000E6E4F9E20081118122813381EEE4F9E2A4
:102080004081518162817381040F151F261F371F04
:1020900043E050E06091952970E0461B570B652F97
:1020A000660F660B762F0E945632EEEEF8E2008342
:1020B000118322833383EEE3F9E2008111812281CF
:1020C0003381E2E5F9E24081518162817381040F3D
:1020D000151F261F371F43E050E06091952970E0DF
:1020E000461B570B652F660F660B762F0E945632E4
:1020F000EAEFF8E20083118322833383EEE5F9E20D
:102100000081118122813381E2E6F9E2408151812F
:1021100062817381040F151F261F371F43E050E0B3
:102120006091952970E0461B570B652F660F660B73
:10213000762F0E945632E6E5F9E20083118322836E
:1021400033830FEF00938B2961C0E2E4F9E2008151
:10215000118122813381EAE4F9E200831183228331
:102160003383E6E4F9E20081118122813381EEE4D8
:10217000F9E20083118322833383EEE3F9E20081E5
:10218000118122813381E2E5F9E200831183228308
:102190003383EEE5F9E20081118122813381E2E6A9
:1021A000F9E2008311832283338330C0EAE2F9E24B
:1021B0000081118122813381E6E3F9E200831183FA
:1021C00022833383EEE2F9E200811181228133819F
:1021D000EAE3F9E20083118322833383E6E2F9E242
:1021E0000081118122813381E2E3F9E200831183CE
:1021F00022833383EEEFF8E2008111812281338163
:10220000EAE5F9E200831183228333835FBE0991FB
:10221000199129913991499159916991799109902F
:10222000199029903990E991F99189919991A99101
:10223000B9914990599018959C01C8010197FC01EA
:10224000CF01EF2BD9F716950795C8010197FC012F
:10225000CF01EF2BD9F7C90108950E94F43400E4AF
:102260000E945102AFEF80E002C0A69583958830AE
:10227000A8F4BA2F90E005C000E00E949502B69540
:102280009395983090F7BB2311F001E001C000E076
:10229000002391F70FE10E949502F1CFE4E00C9446
:1022A00005359A938A9300E40E94510280E008C0A9
:1022B00090E0FC01E455FD4F04910E949502839546
:1022C0008034B0F38991999108950E94F434D80133
:1022D00080E090E02AC00DE210E0AC010E94BD3128
:1022E000F801EA0FFB1FE83601E0F00714F0E856AA
:1022F000F1408F01212F220F220B322F0E94B83282
:1023000045E35AEF6EE87CE30E9478330E946B311C
:10231000AC01440F551F440F551FFA01E25AF74D07
:1023200000831183228333830196883000E0900775
:1023300094F2E4E00C9405350E94F434D80180E076
:1023400090E02AC00DE210E0AC010E94BD31F8011E
:10235000EA0FFB1FE83601E0F00714F0E856F14001
:102360008F01212F220F220B322F0E94B83245E31A
:102370005AEF6EE87CE30E9478330E948E38AC01FD
:10238000440F551F440F551FFA01E25EF74D0083BD
:102390001183228333830196883000E0900794F202
:1023A000E4E00C9405350E94F434D80180E090E01C
:1023B0002AC00DE210E0AC010E94BD31F801EA0F25
:1023C000FB1FE83601E0F00714F0E856F1408F01FA
:1023D000212F220F220B322F0E94B83245E35AEFF1
:1023E0006EE87CE30E9478330E946B31AC01440FAD
:1023F000551F440F551FFA01E25CF74D008311830E
:10240000228333830196883000E0900794F2E4E061
:102410000C9405350E94F034D80180E090E013C0A0
:10242000FC01E95BFC4F049110E0AD010E94BD315D
:10243000000F111F9C01220F331FF901E25FF74DBE
:10244000008311830196883000E090070CF046C0AD
:1024500000917A29002321F70DE210E0AC010E94DF
:10246000BD31A80146535F4F483601E0500714F0D4
:10247000485651408D01212F220F220B322F0E94EE
:10248000B832280139018A01212F220F220B322F65
:102490000E94B83245E35AEF6EE87CE30E9478333D
:1024A0000E948E38A201B3010E94783328013901BD
:1024B0008D01212F220F220B322F0E94B832A20150
:1024C000B3010E9417330E94C5329C01220F331FB3
:1024D000F901E25FF74D00831183B4CFE8E00C947B
:1024E00001350E94EE344801D90180E090E046C0F9
:1024F0000DE210E0AC010E94BD31A801480D591D4C
:10250000483601E0500714F0485651408D01212F04
:10251000220F220B322F0E94B832280139018A0182
:10252000212F220F220B322F0E94B83208011901ED
:1025300045E35AEF6EE87CE3800191010E94783315
:102540000E948E38A201B3010E947833280139011C
:102550008D01212F220F220B322F0E94B832A201AF
:10256000B3010E9417330E94C5329C01220F331F12
:10257000F901E250F84D008311830196883000E0A4
:1025800090070CF4B5CFEAE00C94FF340E94F434C9
:1025900020E030E000E010E0A4DF82D105E00E94FE
:1025A0006203E091D028F091D128F39708F4EDC0B0
:1025B00080E09CE5A1ECB7E400E010E00093AC29DA
:1025C0001093AD2908C0ECEAF9E2008111810B5F9C
:1025D0001F4F008311830091AC291091AD2908365B
:1025E00021E012079CF5209144253091452500916A
:1025F000AC291091AD2975DF02E00E9462030091C1
:10260000D0281091D12820E030E00E94C332AC01E4
:10261000BD010E947A34B8F60091D0281091D128DB
:1026200020E030E00E94C332C801D9010091AC29FA
:102630001091AD290093A8291093A929E091D028E1
:10264000F091D128B89708F0BECF50C080E09CE54B
:10265000A1ECB7E405E010E0F4D000E010E0009356
:1026600044251093452508C0E4E4F5E2008111817A
:10267000025E1F4F00831183009144251091452570
:10268000083E27E0120794F5209144253091452516
:102690000091A8291091A92924DF02E00E94620379
:1026A0000091D0281091D12820E030E00E94C33260
:1026B000AC01BD010E947A34B8F60091D028109187
:1026C000D12820E030E00E94C332C801D901009136
:1026D0004425109145250093AA291093AB29E09138
:1026E000D028F091D128749708F0BECFE091A829A6
:1026F000F091A929349744F0E8EAF9E200811181C8
:102700000350104000831183E091AA29F091AB2976
:102710003B9744F0EAEAF9E2008111810A50104047
:10272000008311832091AA293091AB290091A82917
:102730001091A929D6DE0091AA291091AB29009306
:102740006D2910936E290091A8291091A929009351
:102750006B2910936C2930916C29232F0EE010E027
:102760000E949B0A20916B290FE010E00E949B0AB7
:1027700030916E29232F00E110E00E949B0A2091E6
:102780006D2901E110E00E949B0A0FEF009372296E
:10279000E4E00C9405359A938A93C80100919A2934
:1027A000002351F020939929409194290DE00E9433
:1027B0009F310093982907C000918C29029F0092B5
:1027C0006A0910926B09809366099093670904E087
:1027D0000093400989919991089530918C29329FF5
:1027E00000926A0910926B090093660910936709B9
:1027F00004E00093400908950E94F434D80188E071
:1028000090E018C040918C2950E08C010E94BD31AD
:1028100000936A0910936B09A0936609B093670946
:1028200004E00093400908EE1DEF06DD08EB18E810
:1028300003DD0197813000E0900724F7E4E00C9479
:10284000053520918C2930E0220F331F20936A092F
:1028500030936B0944E650E00E94BD310093660955
:102860001093670904E00093400948E750E00091A5
:10287000C2281091C3280E94EF310E5F0E946203AC
:1028800000E00093400908958A93812F10E0D9DF7A
:1028900000E315E7D1DC082F10E0D3DF899108951C
:1028A00021E631E20EE915E20E94413900E80E947A
:1028B000F10200E310E0C5DF08950E94033140E01B
:1028C00050E064E672E40E9478330E94C5320895B5
:1028D0000E94F034C801D9012A013B0100919629D8
:1028E000002379F4A201B3018C019D010E94033100
:1028F00040E050E064E672E40E9478330E94C53202
:1029000027C0A201B3012A013B010AE010E0209197
:10291000962930E0021B130B212F220F220B322F9E
:102920000E94B832A801B901820193010E94F133DB
:10293000AC01BD010E941733A201B3010E94033113
:1029400040E050E064E672E40E9478330E94C532B1
:102950000B3520E0120714F00BE510E0063A2FEFDC
:10296000120714F405EA1FEFE8E00C9401350E9409
:10297000F034D80122E731E20EE915E20E94413934
:1029800000E80E94F102A13000E0B00714F180E0FD
:10299000082F10E020E030E00E94C3322801390106
:1029A0008D01212F220F220B322F0E94B8320E945C
:1029B0000E35A801B901820193010E947A3478F59D
:1029C000082F07570E9451020EE30E94950283953B
:1029D000DFCF80E008C006E8081B0E9451020CE32C
:1029E0000E9495028395082F10E020E030E00E94BD
:1029F000C332280139010FEF1FEFAD010E94BD3135
:102A0000212F220F220B322F0E94B8320E940E3546
:102A1000A801B901820193010E947A34E0F200E337
:102A200015E70ADCE8E00C9401350E94F434A0E0DC
:102A3000B0E000E00093010204E00E94620380E045
:102A400090E019C0E0E0F2E00081086000830091AE
:102A50002B020023E1F301E000932B02009112020C
:102A600010911302A00FB11F0091A0291091A1296C
:102A7000A01BB10B0196803A00E090071CF300E127
:102A80000093010200E117E2D7DBBB2312F4A0E0C0
:102A9000B0E049E650E08D010E94EF31E4E00C9493
:102AA00005350E94F43480E090E000E000930102DC
:102AB00003E00E946203A0E0B0E013C0E0E0F2E0B7
:102AC00000810860008300912B020023E1F301E004
:102AD00000932B020091120210911302800F911F9C
:102AE0001196A43600E0B0074CF300E10093010218
:102AF00044E650E08C010E94EF31E4E00C9405358F
:102B0000E0E0F2E0008100610083009133020023E5
:102B1000E1F301E0009333024091872950E00091F6
:102B20001402109115020E94D7310895009167296F
:102B30001091682901DC009167291091682933DC24
:102B400000916729109168290093692910936A29D7
:102B50000091692910916A29B8DB089500916729CD
:102B600010916829E9DB00916729109168291BDC25
:102B70000091692910916A29A8DB4091922950E0BF
:102B80000FEF10E00E94BD3145DC0091C22810918A
:102B9000C328009326091093270908959A938A93CE
:102BA00001E010E00E94510A902F80E002E010E066
:102BB0000E94510A10E0802B912B8093C2289093A1
:102BC000C32805E010E00E94510A902F80E006E043
:102BD00010E00E94510A10E0802B912B809367290E
:102BE0009093682907E010E00E94510A902F80E03E
:102BF00008E010E00E94510A10E0802B912B809396
:102C0000692990936A290EE010E00E94510A902FE2
:102C100080E00FE010E00E94510A10E0802B912B21
:102C200080936B2990936C2900E110E00E94510A77
:102C3000902F80E001E110E00E94510A10E0802B0B
:102C4000912B80936D2990936E2903E010E00E94F0
:102C5000510A0093832904E010E00E94510A009376
:102C6000842909EF11E00E94510A0093862907EF99
:102C700011E00E94510A00938F290CE010E00E949D
:102C8000510A009392290DE010E00E94510A00932E
:102C90008E290BEF11E00E94510A009397290CEF47
:102CA00011E00E94510A0093872906EF11E00E946B
:102CB000510A00938C2905EF11E00E94510A0093FC
:102CC00093290DEF11E00E94510A00938D2902E132
:102CD00010E00E94510A009391290AE010E00E943E
:102CE000510A802F90E00BE010E00E94510A102F53
:102CF00000E0802B912B80939C2990939D2903E1E8
:102D000010E00E94510A0093942908EF11E00E94FC
:102D1000510A009378290EEF11E00E94510A0093A6
:102D2000812904E110E00E94510A0093822900E009
:102D300010E00E94510A0093952904EF11E00E94CF
:102D4000510A00937A2903EF11E00E94510A00937F
:102D5000962902EF11E00E94510A00939A29ECE9AA
:102D6000F9E20081016000838991999108950E94A0
:102D7000F434D801AB3500E0B00714F0AAE5B0E0B8
:102D8000BB2312F48CE309C04AE050E08D010E949D
:102D9000EF31102F06E0109F802D00E80E945102B5
:102DA00090E0FC01E451FD4F04910E94950201E87E
:102DB0000E94510290E0FC01E351FD4F04910E94FA
:102DC000950202E80E94510290E0FC01E251FD4FA1
:102DD00004910E94950200EC0E94510290E0FC01D7
:102DE000E151FD4F04910E94950201EC0E945102B5
:102DF00090E0FC01E051FD4F04910E94950202EC2D
:102E00000E94510290E0FC01EF50FD4F04910E949E
:102E10009502BB2312F482E408C04AE050E08D0121
:102E20000E94EF3106E0409F802D04E80E9451028D
:102E300090E0FC01E451FD4F04910E94950205E8E9
:102E40000E94510290E0FC01E351FD4F04910E9469
:102E5000950206E80E94510290E0FC01E251FD4F0C
:102E600004910E94950204EC0E94510290E0FC0142
:102E7000E151FD4F04910E94950205EC0E94510220
:102E800090E0FC01E051FD4F04910E94950206EC98
:102E90000E94510290E0FC01EF50FD4F04910E940E
:102EA000950203E80E94510200E20E94950203ECA1
:102EB0000E94510200E20E949502E4E00C94053564
:102EC0000E94F434ECE9F9E2018107FF02C005E554
:102ED00001C008E53091C72833230AF47BC0209154
:102EE000C6283091C72810E0201731070CF072C0B7
:102EF0004AE050E00091C6281091C7280E94EF31A7
:102F0000402F4A5F00919C2910919D290E94D13148
:102F10000170002309F05EC000918F29013031F467
:102F20002091772900E717E136DCACC000918F29AA
:102F3000023001F5E091C628F091C728759734F466
:102F40002091772900EE1EE226DC9CC00091C62865
:102F50001091C7280B3420E0120734F02091772914
:102F600000EA1FE018DC8EC02091772900E717E106
:102F700012DC88C000918F290330B9F420917729A1
:102F8000A22F8AE090E04AE050E00091C62810911C
:102F9000C7280E94EF31801B910B00E416E0AC01C2
:102FA0000E94BD312A2FF7DB6DC000918F290430BC
:102FB00009F068C02091772904E610E04091C62806
:102FC0005091C728041B150B46E950E00E94BD3103
:102FD000E2DB58C01091C72811230AF053C00091BA
:102FE000842910E020E030E00E94C332C801D901FA
:102FF00003E010E04091C0285091C1280E94BD31EB
:10300000212F220F220B322F0E94B8320E940E3540
:10301000A801B9018C019D010E947A3498F584E0E1
:103020004CEE5FEF0091C6281091C7280E94EF3147
:10303000801B482F00919C2910919D290E94D1311D
:1030400001700023F9F40091C6281091C72800935D
:10305000CA281093CB2800917729009377290091F3
:10306000C6281091C728073E2FEF120734F0209191
:10307000772900E21EE48FDB05C02091772900E666
:103080001DE689DBE4E00C9405359A938A938091E0
:10309000C2289091C3280196AC01652F660F660B7C
:1030A000762F00E01CE62CED32E00E94563243E021
:1030B0000E942B3248E050E060E070E00E94033252
:1030C00040E750E060E070E00E9456320093D6285E
:1030D0001093D72845E00091D6281091D7280E9458
:1030E000CB3140E250E00E94BD310093D6281093CE
:1030F000D7280091D6281091D728000F012F001F44
:1031000010E0111F0093D8281093D928009194291A
:103110000130A9F40091D6281091D7280093D42823
:103120001093D52844E150E00091C2281091C328A3
:103130000E94EF310093DA281093DB2816C000912B
:10314000D6281091D728000F111F0093D428109370
:10315000D5284EE050E00091C2281091C3280E946B
:10316000EF310093DA281093DB2800917E290023A9
:1031700021F400919429033041F400917E29002329
:1031800059F000919429033039F401E010E00093E4
:10319000DC281093DD2806C000E010E00093DC2856
:1031A0001093DD288991999108958A93009181293E
:1031B00010E0F801E65CFC4F0491002359F1009106
:1031C0007C29002339F59CDC2091812930E0F9012C
:1031D000E65CFC4F249130E002171307DCF480E03A
:1031E00017C023E831E20EE915E20E94413900E8F8
:1031F0000E94F10208E710E024DB08EE1DEF0E94B8
:103200001C1101E00E94510202E00E9462038395BA
:10321000853038F38991089510912002137E109320
:1032200020020A95000F000F10912002102B10931E
:1032300020020895B3DC29DF0E941F020091932928
:10324000023039F400917C29002319F40E945111B5
:1032500002C00E942D1120916D2930916E2900919C
:103260006B2910916C293DD979DC00919129D4DF2B
:1032700008952091672930916829201B310B2A5528
:1032800030402093692930936A2910916A291123CB
:1032900042F4E9E6F9E20081118108591E4F0083EA
:1032A00011835CDC30916A29232F07E010E00E9433
:1032B0009B0A2091692908E010E00E949B0A08956A
:1032C0000E94E8342197F89400E30E94F602E0E8B7
:1032D000F6E0008108600083009160060F600093B3
:1032E000600600914006006C00934006E0E6F6E0C0
:1032F000008100620083E0E4F6E000810260008368
:1033000000916006006C0093600608E100931106CE
:1033100008E10093120608E10093130608E1009308
:10332000300608E10093520608E1009353060E941C
:103330001F020AEF11E00E94510A0F3F11F401E051
:1033400001C000E0E8E0F6E0108111FD0CC0E8E00B
:10335000F6E0108112FD07C0E8E2F6E0208121705E
:1033600011E0212701C020E0022B002309F4DEC078
:1033700024E931E20EE915E20E94413900EC0E9495
:10338000F102789402E30E946203F89400E0009353
:10339000A72905C00091A72903950093A7290091AB
:1033A000A729043008F0BDC000E00093A62913C08F
:1033B000B0E0FD01E759FC4F24910A2F10E00054C2
:1033C0001E4F0E949B0AA395A93090F30091A62955
:1033D00003950093A6290091A6290330D8F622E090
:1033E00001E010E00E949B0A27E502E010E00E9445
:1033F0009B0A20E005E010E00E949B0A24EB06E017
:1034000010E00E949B0A20E007E010E00E949B0A67
:1034100020EB08E010E00E949B0A20E00EE010E0A4
:103420000E949B0A20E00FE010E00E949B0A20E02F
:1034300000E110E00E949B0A20E001E110E00E9400
:103440009B0A22E003E010E00E949B0A22E004E0D5
:1034500010E00E949B0A20E009EF11E00E949B0A05
:1034600027E00CE010E00E949B0A21E00DE010E054
:103470000E949B0A21E007EF11E00E949B0A21E0D5
:103480000AE010E00E949B0A20E80BE010E00E9496
:103490009B0A20E00BEF11E00E949B0A28E10CEF51
:1034A00011E00E949B0A27E006EF11E00E949B0AB0
:1034B00026E00DEF11E00E949B0A22E002E110E0FD
:1034C0000E949B0A21E005EF11E00E949B0A21E087
:1034D00003E110E00E949B0A20E008EF11E00E9447
:1034E0009B0A22E00EEF11E00E949B0A24E004E117
:1034F00010E00E949B0A21E000E010E00E949B0A7D
:1035000020E004EF11E00E949B0A20E003EF11E0AD
:103510000E949B0A21E002EF11E00E949B0AA0E0BA
:1035200053CF20E00AEF11E00E949B0A0AEF11E05E
:103530000E94510A0093A72900E00093A6297ADE91
:1035400000919A29033018F001E000939A29209104
:103550009A2902EF11E00E949B0A03E0009384295C
:1035600002E00093832903E20093010807E000933F
:10357000000806E910E000932608109327088091C0
:103580008D2990E0019680932A0890932B08009152
:103590008D29002331F400E010E0009326081093F9
:1035A000270801E0009300090091C2281091C32868
:1035B000009326091093270903E000930609009160
:1035C000A20007600093A20007E00093400804ED0A
:1035D00011E0009366081093670801E00093460825
:1035E0000E94480320916D2930916E2900916B292A
:1035F00010916C290E9471120E941F0302E0009337
:1036000022020E9441030E943A030E941F0300917C
:10361000912902DEA3DA02E00E94620342DA0093FB
:10362000A0291093A12903E20093410900916406A7
:103630000F730093640626EA31E20EE915E20E9458
:10364000413900EC0E94F10200E210E01A930A9363
:1036500027EB31E20EE915E20E944139229600E89B
:103660000E94F10200ED17E00E94FC1300EA1FE047
:103670000E94FC1300E41FE10E94FC1308EE1DEF02
:103680000E941C1100ED17E00E94FC1300E0009363
:1036900040090091DA28102F06E0109F002D0E94AB
:1036A000620300E61AEE0E941C1100919E250B3465
:1036B00009F0B9CF00919F25003509F0B4CF0091F2
:1036C000A0250F3409F0AFCF00918629002331F0F7
:1036D000009164060F730093640605C000916406B0
:1036E000006C009364060091A125043509F09BCF7E
:1036F0008091A72990E001969A938A932AEC31E26F
:103700000EE915E20E944139229600EC0E94F10276
:1037100007EC0E945102A0E009C00A2F10E00054FB
:103720001E4F0E94510A0E949502A395A930A8F34A
:103730000091DA28102F05E0109F002D0E946203EF
:1037400078940CE00E94510202E00E9462032DDD99
:10375000E8E0F6E0008101FD24C0E8E0F6E0008149
:1037600002FD1FC00FEF00937C2901E000937B292D
:1037700001E000937D2901E00E94510210E500E381
:103780000E94441423ED31E20EE915E20E94413912
:1037900000E80E94F102E8E0F6E0008102FFFBCFC2
:1037A0006EC1E8E0F6E0008102FD21C00FEF00935A
:1037B0007C2906E000937B2902E000937D2901E04B
:1037C0000E94510210E500E30E94441424EE31E20D
:1037D0000EE915E20E94413900E80E94F102E8E09A
:1037E000F6E0008102FFFBCF0E942D1148C100E0EE
:1037F00000937D2900E61AEE0E941C1116D93801AB
:10380000A091DA2860C04091C2285091C3284F5F30
:103810005F4F652F660F660B762F00E01CE62CEDE0
:1038200032E00E94563243E00E942B32C8017A9265
:103830006A929A938A932FE132E20EE915E20E948E
:103840004139249600E80E94F1020091D02810919D
:10385000D1281A930A932EE232E20EE915E20E9471
:103860004139229600EC0E94F1020091942910E067
:10387000000F111FF801E35BFC4F059114911A939F
:103880000A930091952910E01A930A9300919129C7
:1038900010E0F801E15CFC4F049110E01A930A93E8
:1038A0002AE332E20EE915E20E944139269609EC3C
:1038B0000E94F1020FEC0E9451020AE20E9495025E
:1038C00003E00E9462030A2FA02FAA95002309F0AB
:1038D00055C001E00E94510200E21EE40E941C114A
:1038E00005E0601600E070060CF088C024E432E2C7
:1038F0000EE915E20E94413900E80E94F10200ED54
:1039000010E00E94211400EB10E00E94211400ED51
:1039100010E00E94211404E10E946203B0C081E023
:1039200090E00091952910E01A930A930091912953
:1039300010E0F801E15CFC4F049110E01A930A9347
:1039400000916729109168292091692930916A298D
:10395000021B130B1A930A939A938A93B0E0BA93BB
:10396000AA9328E032E20EE915E20E9441392A9634
:1039700000EC0E94F10208E00E946203E8E2F6E037
:10398000008100FD40CF0AE00E9462038090D028B1
:103990009090D1280091902910E01A930A937A927E
:1039A0006A929A928A9225EF31E20EE915E20E941C
:1039B0004139269600E80E94F10200919C2910915D
:1039C0009D29013020E8120761F000E020919C2938
:1039D00030919D29213010E0310719F0006000235B
:1039E00011F0A0E001C0A1E000916D2910916E29B5
:1039F000012B09F094CF80E090E093CF0091D02884
:103A00001091D128093522E01207C8F10091D02881
:103A10001091D1281A930A9322E532E20EE915E2B9
:103A20000E944139229603E80E94F1022CE532E21D
:103A30000EE915E20E94413900EC0E94F10200ED0E
:103A400010E00E94211400EB10E00E94211400ED10
:103A500010E00E942114A1E010C008EE1DEF0E94AA
:103A60001C11E8E0F6E0008102FD06C00E94C612CB
:103A700010E200E30E944414A395A23370F300E027
:103A80000093882902E30093802900937F2900E0B6
:103A900010E020E030E0E2E2F9E2008311832283CB
:103AA0003383E6E1F9E200831183228333830093B9
:103AB000CA281093CB280093C8281093C928212F17
:103AC000220F220B322FEAEFF8E2008311832283C8
:103AD000338301E010E000939E2910939F2904E0B6
:103AE0000E94620300E310E00E94211401E00093B1
:103AF000732903E00E94620300E310E00E94211496
:103B000020C000916406006C0093640600E20093FC
:103B1000662901E0E00E00E0F01E87017801013423
:103B20002FE1120774F0EE24FF243FDB0091D02830
:103B30001091D128083E23E0120718F401E0009309
:103B4000732900917C29002309F065C40091DC28C9
:103B50001091DD28013020E0120709F0D1C1EAEE12
:103B6000F8E20081118122813381EEE0F9E20083E5
:103B7000118322833383EEEEF8E2008111812281EA
:103B80003381EAE1F9E20083118322833383EAEF90
:103B9000F8E2008111810093C0281093C12842E00F
:103BA00050E060E070E0E6E5F9E2008111812281F9
:103BB00033810E94563200936F291093702900912F
:103BC00083290D5F10918E29011B00938529009197
:103BD000852910E02091C0283091C12802171307D1
:103BE0000CF02DC100917B29002309F028C100E0D1
:103BF00000937F29009180290395009380290091EB
:103C00008029003118F001E000937329E2E1F9E224
:103C10000081118122813381EEE0F9E240815181FE
:103C200062817381401B510B620B730B4083518384
:103C300062837383EEE1F9E2008111812281338195
:103C4000EAE1F9E24081518162817381401B510BAD
:103C5000620B730B4083518362837383EEE0F9E25E
:103C60000081118122813381EEE0F9E240815181AE
:103C7000628173810E940332C801D901EAE1F9E24D
:103C80000081118122813381EAE1F9E24081518191
:103C9000628173810E940332A801B9018C019D01E8
:103CA000040F151F261F371F0E94B8320E945C396F
:103CB0000E94C53228015594479455944794552045
:103CC0004AF428E004EF1EE70E94CB1300E21EE452
:103CD0000E941C11EAE1F9E2008111812281338105
:103CE0000E94B832A801B901CA01DB01EEE0F9E295
:103CF00000811181228133810E94B832AC01BD0163
:103D00000E9468140093C6281093C7280091802948
:103D1000043048F1E091C628F091C728B9971CF10A
:103D2000E091C028F091C1283A97ECF0E6EFF8E274
:103D300000811181228133810E94B832A801B9012A
:103D4000CA01DB01E2EFF8E20081118122813381B7
:103D50000E94B832AC01BD010E945D140093C428DA
:103D60001093C52806C000E010E00093C42810930B
:103D7000C5280091C0281091C1280F5F1F4F212F27
:103D8000220F220B322F0E94B8320E940E350E9461
:103D9000C5320093772900917829002321F408E0A7
:103DA0000093772917C000917829013041F40091E0
:103DB000772910917729100F109377290BC0009164
:103DC0007829023039F40091772910917729019FE1
:103DD000009277290091772910E049E050E0209186
:103DE0008C2930E0421B530B0E94EF310395009366
:103DF00077290091C0281091C128C016D10684F4FB
:103E00000091C6281091C7280093CC281093CD2884
:103E100040929E2950929F29C090C028D090C128DE
:103E20000091CC281091CD280093CA281093CB285C
:103E30000093C6281093C7280E946017ECC2009117
:103E40009A29002331F400E010E000936A091093EE
:103E50006B09EEE0F9E20081118122813381E2E118
:103E6000F9E20083118322833383EAE1F9E20081DE
:103E7000118122813381EEE1F9E2008311832283F3
:103E80003383CC24DD2400917F29039500937F297F
:103E900000E00093802900919A29023009F0BBC20A
:103EA0002091832930E000918E2910E0200F311FEE
:103EB00000916F29109170292017310794F4009117
:103EC0009829002371F400919B29039500939B2965
:103ED000043008F4A0C222E000E516E40E94ED13CD
:103EE0009AC200E000939B2900919829002309F0D1
:103EF00092C200E010E000936A0910936B098BC234
:103F000000917E29002309F01BC100919429033000
:103F100009F016C1EAEEF8E20081118122813381B5
:103F2000E6E1F9E24081518162817381041B150B46
:103F3000260B370BEEE0F9E20083118322833383F3
:103F4000EEEEF8E20081118122813381E2E2F9E2B2
:103F50004081518162817381041B150B260B370B45
:103F6000EAE1F9E20083118322833383EAEFF8E286
:103F7000008111810093C0281093C128EEEEF8E271
:103F800000811181228133810E94B832A801B901D8
:103F9000CA01DB01EAEEF8E200811181228133815E
:103FA0000E94B832AC01BD010E9468140093C6287B
:103FB0001093C7280091C6281091C728053A2FEF03
:103FC000120761F000E02091C6283091C7282B35F8
:103FD00010E0310719F00060002341F00091CA2879
:103FE0001091CB280093C6281093C728EEE0F9E281
:103FF0000081118122813381EEE0F9E2408151811B
:10400000628173810E940332C801D901EAE1F9E2B9
:104010000081118122813381EAE1F9E240815181FD
:10402000628173810E940332A801B9018C019D0154
:10403000040F151F261F371F0E94B8320E945C39DB
:104040000E94C53245E00E94D131280155204AF432
:1040500027E000E01DE70E94CB1300E41CE90E946A
:104060001C11088103950883003128F001E00093BA
:10407000732900E0088300917829002321F408E0E7
:104080000093772907C00091772910917729100FA5
:10409000109377290091772910E049E050E02091B2
:1040A0008C2930E0421B530B0E94EF3103950093A3
:1040B0007729042D052939F442E0009177290E94DF
:1040C0009F310093772904E00093400900918C29E7
:1040D000069510917729019F00926A0910926B0949
:1040E000E091C028F091C1283197ECF0E091C6280A
:1040F000F091C72831976CF000E41FE12091C028AF
:104100003091C128021B130B0093660910936709B5
:104110000AC00091C0281091C128005C104E009385
:1041200066091093670940929E2950929F29009139
:10413000C6281091C7280093CA281093CB286BC1BA
:1041400042E050E060E070E0EAEEF8E200811181C8
:10415000228133810E945632EEE0F9E2008311831E
:104160002283338342E050E060E070E0EEEEF8E25C
:1041700000811181228133810E945632EAE1F9E205
:10418000008311832283338342E050E060E070E0DB
:10419000EAEFF8E200811181228133810E945632D8
:1041A0000093C0281093C128EEE0F9E2008111814C
:1041B00022813381EEE0F9E2408151816281738195
:1041C0000E940332C801D901EAE1F9E200811181BC
:1041D00022813381EAE1F9E2408151816281738178
:1041E0000E940332A801B9018C019D01040F151F23
:1041F000261F371F0E94B8320E945C390E94C532C8
:1042000043E00E94D13128010091832910E02091E0
:10421000C0283091C128021713070CF0D7C00091B5
:104220007B29002309F0D2C000E000937F29009190
:104230008029039500938029E2E1F9E20081118150
:1042400022813381EEE0F9E2408151816281738104
:10425000401B510B620B730B40835183628373834A
:10426000EEE1F9E20081118122813381EAE1F9E294
:104270004081518162817381401B510B620B730B32
:104280004083518362837383EAE1F9E20081118103
:10429000228133810E94B832A801B901CA01DB0131
:1042A000EEE0F9E200811181228133810E94B8326F
:1042B000AC01BD010E9468140093C6281093C72862
:1042C00055204AF427E000E01DE70E94CB1300E4EC
:1042D0001CE90E941C110091C0281091C1280F5F99
:1042E0001F4F212F220F220B322F0E94B8320E9423
:1042F0000E350E94C532009377290091782900235A
:1043000021F408E00093772917C000917829013043
:1043100041F40091772910917729100F1093772994
:104320000BC000917829023039F40091772910915F
:104330007729019F009277290091772910E049E0C1
:1043400050E020918C2930E0421B530B0E94EF314A
:1043500003950093772900918029043098F02091EB
:104360007729A22F80EE9EE242E050E00091C02823
:104370001091C1280E94EF31801B910B8C012A2FD4
:104380000E94CB130091C0281091C128C016D106FD
:1043900084F40091C6281091C7280093CC2810936C
:1043A000CD2840929E2950929F29C090C028D0903D
:1043B000C1280091CC281091CD280093CA281093D1
:1043C000CB280093C6281093C72825C000E000938F
:1043D0004009EEE0F9E20081118122813381E2E1BE
:1043E000F9E20083118322833383EAE1F9E2008159
:1043F000118122813381EEE1F9E20083118322836E
:104400003383CC24DD2400E00093802900917F29B0
:10441000039500937F2900917F29003F41F010E030
:1044200000918029003F19F010601123A9F000E0ED
:1044300010E000939E2910939F290093CA2810939F
:10444000CB280093C8281093C9280093C428109340
:10445000C52801E00093732900917B29E2E7F3E08E
:104460000C94A3348091CA289091CB28E0919E2986
:10447000F0919F2934972CF08093C8289093C928F5
:1044800004C08091C8289091C928009193290230D6
:1044900009F093C08C010E94B71604E610E00E9458
:1044A0001C1100919E2910919F29212F220F220B70
:1044B000322F0E94B8320E940E350E94C532C801C8
:1044C00000917F29053048F02DE632E20EE915E231
:1044D0000E94413907EC0E94F102552032F403E2B8
:1044E000802E992489E090E00DC00091DC28109185
:1044F000DD28012B21F40EE3802E992403C006E071
:10450000802E9924A0E008C00A2F08530E9451026F
:10451000082D0E949502A395B0E0A817B907A4F34F
:104520000091662910E01A930A9300918E2910E0F9
:104530001A930A930091832910E01A930A93009129
:10454000842910E01A930A9327E732E20EE915E274
:104550000E944139289607E80E94F1020E948015C6
:1045600048014AE050E084010E94EF315A934A9397
:104570004AE050E084010E94EF311A930A9322E846
:1045800032E20EE915E20E94413924960DE80E94BC
:10459000F1020091C4281091C528013F2FEF1207A6
:1045A0000CF061C507E80E94510201E20E949502E9
:1045B00000E117E20E941C1156C5992352F09A930C
:1045C0008A9329E832E20EE915E20E9441392296E7
:1045D0000EC04FEF5FEF8C010E94BD311A930A931A
:1045E00020E932E20EE915E20E944139229600E804
:1045F0000E94F10200919E2910919F29212F220FE4
:10460000220B322F0E94B8320E940E350E94C53212
:10461000C80199231AF483E290E006C0883000E0D4
:10462000900711F48FEF90E004E80E945102082FE8
:104630000E9495020091662910E01A930A93009156
:104640008E2910E01A930A930091832910E01A939F
:104650000A930091842910E01A930A9327E932E221
:104660000EE915E20E944139289605E80E94F10200
:104670000E94801548014AE050E084010E94EF3119
:104680005A934A934AE050E084010E94EF311A9312
:104690000A9324EA32E20EE915E20E944139249697
:1046A0000DE80E94F1020091C4281091C528013F35
:1046B0002FEF120754F406E80E94510201E20E9413
:1046C000950200E117E20E941C110091DC28109174
:1046D000DD28013020E0120709F04FC000917F294A
:1046E000063048F02AEA32E20EE915E20E9441392A
:1046F00000EC0E94F102E091C628F091C7283197A2
:104700007CF00091C6281091C728045C1F4F4AE036
:1047100050E00E94EF310093CE281093CF2812C0B2
:1047200042E050E00091C6281091C7280E94EF3166
:104730000E5C1F4F4AE050E00E94EF310093CE28FC
:104740001093CF280091CE2800540E94510282304D
:1047500000E090075CF000917F29013020F006E036
:104760000E94950203C004E00E94950205EC0E949D
:1047700051020FE20E94950276C443E082010E943A
:10478000D131C801833C01E0900734F400E0992363
:104790001AF00060002311F082EC91E02BEB32E282
:1047A0000EE915E20E94413900EC0E94F102A0E0FE
:1047B0000FC00A2F07530E9451020EE30E94950278
:1047C00006EC0A1B0E9451020CE30E949502A3957D
:1047D0000A2F10E020E030E00E94C3324801590166
:1047E0008C01212F220F220B322F0E94B8320E94FF
:1047F0000E35A801B901840195010E947A34C8F2EE
:1048000000ED17E00E941C112EC48091A72990E0B2
:1048100001969A938A932CEC32E20EE915E20E94FB
:104820004139229600E80E94F10207E80E945102F5
:10483000A0E009C00A2F10E000541E4F0E94510A48
:104840000E949502A395A930A8F300E21EE40E94FD
:104850001C11E8E2F6E0008100FD6CC008E210E007
:104860000E9421140DE00E945102A0E407E0009391
:1048700088290FC000918829039500938829003169
:1048800018F00FE000938829A0E408E210E00E94ED
:1048900021140091882900580E94510206E00E94CC
:1048A0006203E8E0F6E0008102FFE4CFE8E0F6E032
:1048B000008101FD10C0009188290A950093882984
:1048C000073018F407E000938829A0E408E210E01C
:1048D0000E942114DECFE8E2F6E0008100FD1EC058
:1048E000A3950A2FA02F0B3508F0A0E3AA3309F4F3
:1048F000A0E20A2F0E9495020091882900580E9488
:10490000510202E310E00E9421142A2F009188290D
:1049100010E007541E4F0E949B0ABBCFE8E0F6E070
:10492000008103FDB6CF08E210E00E9421140CE0E4
:104930000E9451020E942D1125ED32E20EE915E28E
:104940000E94413900EC0E94F102A0E010C00A2F41
:104950000A530E9451020A2F0E949502A83031F496
:104960000EEC0E9451020FEF0E949502A3958091D8
:10497000A72990E00196B0E08A179B0744F773C31C
:104980000E948015C8014AE050E08C010E94EF317E
:104990005A934A934AE050E08C010E94EF311A93F7
:1049A0000A930091812910E0F801E65CFC4F049124
:1049B0004AE00E949F3150E05A934A930091812926
:1049C00010E0F801E65CFC4F04914AE00E949F3140
:1049D00010E01A930A9326EE32E20EE915E20E94E5
:1049E0004139289600E80E94F1020091872910E0E1
:1049F0001A930A932CEF32E20EE915E20E94413934
:104A0000229600EC0E94F10202E00E9462032BC396
:104A100000918D2910E01A930A932DE033E20EE9FC
:104A200015E20E944139229600E80E94F1022FE12E
:104A300033E20EE915E20E94413900EC0E94F102D6
:104A4000A0E010C00A2F0A530E9451020A2F0E94B0
:104A50009502A83031F40EEC0E9451020FEF0E9433
:104A60009502A39500918D290A1760F702E00E9434
:104A70006203F9C20E941515C8019A938A9321E333
:104A800033E20EE915E20E944139229600E80E94C5
:104A9000F1020091D4281091D5281A930A9324E4A6
:104AA00033E20EE915E20E944139229609E80E949C
:104AB000F1024091C2285091C3284F5F5F4F652F8C
:104AC000660F660B762F00E01CE62CED32E00E94AC
:104AD000563243E00E942B323A932A931A930A9358
:104AE0002DE433E20EE915E20E944139249600ECF0
:104AF0000E94F10200E21EE40E941C11B4C240E2D6
:104B000050E060E070E0EEEEF8E200811181228179
:104B100033810E9456320E94B7142DE533E20EE92C
:104B200015E20E94413900EC0E94F1020FED10E005
:104B30001A930A9300916729109168291A930A938E
:104B400028E633E20EE915E20E94413924960AEC88
:104B50000E94F10200E21EE40E941C1184C2009136
:104B60007A29002311F4A3E501C0ADE40E941515D4
:104B70001A930A9321E733E20EE915E20E944139C4
:104B8000229600E80E94F102B0E0BA93AA9329E7C6
:104B900033E20EE915E20E944139229606E80E94AE
:104BA000F10225E833E20EE915E20E94413900ECFA
:104BB0000E94F102A0E010C00A2F0A530E94510285
:104BC0000A2F0E949502A83031F40EEC0E94510287
:104BD0000FEF0E949502A395009192290A1760F7A2
:104BE00002E00E9462033FC20091952910E01A93EF
:104BF0000A930091912910E0F801E15CFC4F0491C7
:104C000010E01A930A9326E933E20EE915E20E94B6
:104C10004139249600E80E94F1022FE933E20EE9BF
:104C200015E20E94413906E80E94F1022AEA33E2C5
:104C30000EE915E20E94413900EC0E94F102A0E069
:104C400010C00A2F0A530E9451020A2F0E94950297
:104C5000A83031F40EEC0E9451020FEF0E94950231
:104C6000A395009191290A1760F702E00E94620360
:104C7000FAC10091D0281091D1281A930A932BEBF6
:104C800033E20EE915E20E944139229600E80E94C3
:104C9000F10200916D2910916E291A930A9326EC66
:104CA00033E20EE915E20E944139229609E80E949A
:104CB000F1020FED10E01A930A9300916B29109105
:104CC0006C291A930A932FEC33E20EE915E20E9445
:104CD0004139249600EC0E94F102009172290023D0
:104CE00021F409E80E94510203C009EC0E9451021C
:104CF0000EE30E94950202E00E946203B4C100919B
:104D0000822910E01A930A9322EE33E20EE915E2AB
:104D10000E944139229600E80E94F1022FE933E215
:104D20000EE915E20E94413906E80E94F1022AEEDE
:104D300033E20EE915E20E94413900EC0E94F102D3
:104D4000A0E010C00A2F0A530E9451020A2F0E94AD
:104D50009502A83031F40EEC0E9451020FEF0E9430
:104D60009502A395009182290A1760F702E00E943C
:104D7000620379C144E050E060E070E0EAEFF8E2FD
:104D800000811181228133810E9456320E94B71422
:104D90002BEF33E20EE915E20E94413900EC0E944C
:104DA000F1020FED10E01A930A9300916929109116
:104DB0006A291A930A9328E633E20EE915E20E9463
:104DC000413924960AEC0E94F10200E41CE90E9499
:104DD0001C1149C10091782910E0000F111FF80142
:104DE000EB5AFC4F059114911A930A9327E034E291
:104DF0000EE915E20E944139229600E80E94F10274
:104E00002FE933E20EE915E20E94413906E80E94DB
:104E1000F1022EE034E20EE915E20E94413900EC85
:104E20000E94F102A0E010C00A2F0A530E94510212
:104E30000A2F0E949502A83031F40EEC0E94510214
:104E40000FEF0E949502A39500918C290A1760F735
:104E500000E61AEE0E941C1106C100918F29033052
:104E600019F48AE090E00CC000918F29043019F405
:104E70008AE590E005C080918F2990E0880F991F06
:104E80009A938A932FE134E20EE915E20E944139A8
:104E9000229600E80E94F10200919A2910E0000F8A
:104EA000111FF801E55AFC4F059114911A930A93CA
:104EB00028E234E20EE915E20E944139229607E821
:104EC0000E94F10221E334E20EE915E20E94413929
:104ED00000EC0E94F102A0E008C00A2F06530E94D5
:104EE00051020A2F0E949502A39500918F290A175B
:104EF000A0F702E00E946203B6C00091962910E07C
:104F00001A930A930091932910E0000F111FF801E2
:104F1000E15AFC4F059114911A930A9322E434E26A
:104F20000EE915E20E944139249600E80E94F10240
:104F300022E534E20EE915E20E94413900EC0E94BC
:104F4000F102A0E010C00A2F0A530E9451020A2F5A
:104F50000E949502A83031F40EEC0E9451020FEF2E
:104F60000E949502A395009196290A1760F702E026
:104F70000E94620378C00091942910E0000F111F75
:104F8000F801E35BFC4F059114911A930A9323E611
:104F900034E20EE915E20E944139229600E80E94AF
:104FA000F10221E734E20EE915E20E94413900ECFA
:104FB0000E94F102A0E010C00A2F0A530E94510281
:104FC0000A2F0E949502A83031F40EEC0E94510283
:104FD0000FEF0E949502A395009194290A1760F79C
:104FE00002E00E94620301E0009375293CC0009139
:104FF00075290023C1F123E834E20EE915E20E948D
:10500000413900E80E94F102A0E004C000E20E94E1
:105010009502A395A03190F40A2F00540E945102EA
:105020004A2F00919C2910919D290E94D131017035
:10503000002361F303E20E949502EBCF05EC0E948E
:1050400051020FE20E9495020091882900540E94AB
:1050500051020EE00E94510200E00093752908EE13
:105060001DEF0E941C11B0E0E8E0F6E0008103FDB6
:10507000C7C000E00093400901E00093732900914C
:1050800079290130B1F406E210E00E942114E8E031
:10509000F6E0008103FFFBCF01E00093732904EBEE
:1050A0000093802900937F2900E0009379290C94D4
:1050B000F030E8E0F6E0008103FD54C008EE1DEF9B
:1050C0000E941C11B3950B2FB02F2091DA2830913C
:1050D000DB2810E02017310760F700917C2900954C
:1050E00000937C2901E000937929009193290230F3
:1050F00019F40E94511102C00E942D1101E00E947A
:10510000510200917C29002381F400E000937B2967
:105110004091922950E00FEF10E00E94BD310E94B3
:105120000A1202E00E9462030CC00BE000937B298C
:1051300002E00E94620300E010E00E940A120E9456
:105140002D1101E00093752900E000937D2900E016
:1051500000937E290AE510E00E94211401E00093EB
:105160007329A9C100917C29002369F400917E294B
:10517000009500937E290E94451804EB0093802936
:1051800000937F2938C00CE00E94510200917D29D4
:10519000013059F400917B29039500937B290B3052
:1051A000E8F001E000937B2919C000917D290230CD
:1051B00059F400917B29039500937B290B3070F003
:1051C00006E000937B290AC000917B290395009398
:1051D0007B29003118F001E000937B2900917B29A5
:1051E0000C3049F44091922950E00FEF10E00E94FA
:1051F000BD310E940A1208E210E00E942114EDC79E
:10520000E8E2F6E0008100FDB6C300E0009340094B
:1052100000917B29E8E9F3E00C94A33401E00E94BB
:10522000510200E21EE40E941C11E8E2F6E0008157
:1052300000FD0FC008EE1DEF0E941C11B3950B2F4F
:10524000B02F2091DA283091DB2810E020173107A9
:1052500060F7B3950B2FB02F2091DA283091DB281F
:1052600010E02017310708F072C0E6EFF8E2008185
:105270001181228133810E94B832A801B901CA018B
:10528000DB01E2EFF8E200811181228133810E948B
:10529000B832AC01BD010E9468140093C628109377
:1052A000C728E2EFF8E20081118122813381E6E133
:1052B000F9E20083118322833383E6EFF8E2008171
:1052C000118122813381E2E2F9E20083118322839A
:1052D00033830091C6281091C7280F3C2FEF120787
:1052E00064F400E02091C6283091C728263A1FEFC9
:1052F00031071CF00060002391F024E934E20EE94C
:1053000015E20E94413900EC0E94F10200EA10E02F
:105310000E94211400EB10E00E9421146CC025EAC9
:1053200034E20EE915E20E94413900EC0E94F102DC
:105330000091C6281091C7280E94391900E510E095
:105340000E94211400E210E00E94211454C001E0E8
:10535000009373290091D0281091D1281A930A93B1
:1053600026EB34E20EE915E20E944139229600E86C
:105370000E94F10200E310E00E94211400918029B4
:10538000002311F401E001C000E000937F2908E050
:105390000E94620322C78201212F220F220B322F8B
:1053A0000E94B8320E940E354091C6285091C728FD
:1053B0005A934A9340E050E060E070E40E947833F2
:1053C0000E94C5321A930A9328EC34E20EE915E2E2
:1053D0000E944139249600E80E94F10222E000E494
:1053E0001FE1E6E5F9E240815181440F551F041B9E
:1053F000150B0E94CB13E8E2F6E0008100FD4CC0E3
:10540000E8E0F6E0008102FD15C0E6ECF8E200817C
:1054100011810F5F1F4F008311830091C6281091E7
:10542000C7280E94391900E410E00E94211406E008
:105430000E946203E8E0F6E0008101FD15C0E6ECA1
:10544000F8E2008111810150104000831183009126
:10545000C6281091C7280E94391900E410E00E9464
:10546000211406E00E946203E8E0F6E0008103FDFB
:1054700092CF00E310E00E94211425EA34E20EE905
:1054800015E20E94413900EC0E94F1020091C62809
:105490001091C7280E94391900E0009340090AE0E2
:1054A0000E9462032DED34E20EE915E20E944139BB
:1054B00000EC0E94F10291C60091812903950093AE
:1054C0008129053018F000E000938129209181297D
:1054D0000EEF11E00E949B0A0091DA281091DB2860
:1054E0000E941C1102E310E00E94211476C6A0E085
:1054F000B0E00E9450148DE591E012C0809326091F
:105500009093270904E00E9462030E941515A017DA
:10551000B1072CF4D8018093C2289093C328049635
:10552000873E03E0900754F30091C2281091C328EE
:1055300000932609109327090E94451810E400E5FE
:105540000E9444143091C328232F01E010E00E94F0
:105550009B0A2091C22802E010E00E949B0A3DC6EF
:1055600020E135E20EE915E20E94413900E80E948F
:10557000F10200E810E00E94211400E810E00E940F
:105580002114E8E2F6E0008100FDE9C000E61AEE31
:105590000E941C11B3950B2FB02F2091DA28309167
:1055A000DB2810E02017310760F701E0009376292F
:1055B0002EEE34E20EE915E20E94413900E80E9425
:1055C000F10200E310E00E94211401E0009373292E
:1055D00002E30E9462032FEF34E20EE915E20E941B
:1055E000413900E80E94F10200E310E00E9421141A
:1055F00008E20E94620380E090E0A0E01EC0E6EFB7
:10560000F8E200811181228133810E94B832A80121
:10561000B9014A015B01E2EFF8E2008111812281C8
:1056200033810E94B832A401B5010E945D14800F3D
:10563000911F08E00E946203A395AA3000F34AE09C
:1056400050E08C010E94EF31C801E0916729F09190
:105650006829EA55F040E81BF90BE0936729F093BD
:1056600068290091672910916829093621E01207FD
:1056700044F0E7E6F9E20081118108561140008309
:10568000118310916829112342F4E7E6F9E20081C1
:10569000118108591E4F008311830E9496150091B5
:1056A000DA280E946203E6EFF8E20081118122818C
:1056B00033810E94B832A801B9014A015B01E2EFCF
:1056C000F8E200811181228133810E94B832A40165
:1056D000B5010E945D1448010CEA80160FEF900698
:1056E0000CF03ECF21E235E20EE915E20E9441398D
:1056F00000E80E94F10205E210E00E94211405E09A
:105700000E94620305E210E00E94211400916729C3
:10571000109168290093692910936A2900916929D9
:1057200010916A290E94651130916829232F05E0A4
:1057300010E00E949B0A2091672906E010E00E9479
:105740009B0A30916A29232F07E010E00E949B0AF0
:105750002091692908E010E00E949B0A12CF009175
:105760007629002389F422E335E20EE915E20E944E
:10577000413900E80E94F10208EE1DEF0E941C1161
:1057800000E510E00E94211428C500917A29002329
:1057900021F401E000937A2903C000E000937A2904
:1057A0004091922950E00FEF10E00E94BD310E941D
:1057B0000A1220917A2904EF11E00E949B0A02E369
:1057C00010E00E94211404E00E94620306C50091CB
:1057D0009529039500939529033018F001E0009373
:1057E00095292091952900E010E00E949B0A02E390
:1057F00010E00E94211404E00E946203EEC4E8E27B
:10580000F6E0008100FD1AC008EE1DEF0E941C1199
:10581000B3950B2FB02F2091DA283091DB2810E0C0
:105820002017310760F700E610E00E9421140E9463
:10583000C61210E200E30E944414CFC40091722902
:1058400000950093722902E310E00E94211405E004
:105850000E946203C2C400917829039500937829BD
:10586000033018F000E0009378292091782908EFA0
:1058700011E00E949B0A02E310E00E941C1102E367
:1058800010E00E942114A9C400919A290395009365
:105890009A29033018F000E000939A2920919A2960
:1058A00002EF11E00E949B0A02E310E00E94211423
:1058B00008E00E94620391C400919329039500932C
:1058C0009329033018F001E0009393292091932944
:1058D00005EF11E00E949B0A02E310E00E942114F0
:1058E00004E00E94620379C481E090E0409188293D
:1058F0008C010E94C531C8014091882900919C29E2
:1059000010919D290E94D1310170002379F080957A
:105910009095ECE9F9E200811181082319230083B5
:10592000118310E500E40E9444140CC0ECE9F9E294
:1059300000811181082B192B0083118310E300E4EF
:105940000E94441401E00093752920919C290AE0EB
:1059500010E00E949B0A30919D29232F0BE010E05C
:105960000E949B0A3AC401E00093732908E210E008
:105970000E94211432C4E8E0F6E0008102FD1EC25C
:1059800000E00093400900917B29EEEBF3E00C94DA
:10599000A334E8E0F6E0008102FD25C000E61AEE3F
:1059A0000E941C11B3950B2FB02F2091DA28309153
:1059B000DB2810E02017310760F700918629009559
:1059C000009386292091862909EF11E00E949B0A05
:1059D00001E00093762900E510E00E94211401E027
:1059E0000E946203FDC300917629002381F4009197
:1059F00083290395009383290A3018F000E000936F
:105A000083292091832903E010E00E949B0ACEC1E4
:105A10000091A72903950093A729043018F003E00B
:105A20000093A7290E941A192091A7290AEF11E0D3
:105A30000E949B0ABBC10091872903950093872987
:105A40000D3318F001E000938729209187290CEF8E
:105A500011E00E949B0A00E41CE90E941C11A6C1EF
:105A600000918D29039500938D29093018F008E0E5
:105A700000938D290BE910E0009326081093270866
:105A800020918D290DEF11E00E949B0A80918D29B4
:105A900090E0019680932A0890932B0887C180910B
:105AA000C2289091C32801978093C2289093C3285D
:105AB0008D3501E0900734F40DE511E00093C22824
:105AC0001093C3280091C2281091C328009326097F
:105AD000109327090E9445183091C328232F01E015
:105AE00010E00E949B0A2091C22802E010E00E9470
:105AF0009B0A5CC1809167299091682901968093E7
:105B0000672990936829883601E0900734F000E017
:105B100010E000936729109368290E949615009160
:105B20006729109168290093692910936A29309197
:105B30006829232F05E010E00E949B0A2091672925
:105B400006E010E00E949B0A31C100919229039562
:105B500000939229093018F008E0009392294091AF
:105B6000922950E00FEF10E00E94BD310E940A120E
:105B7000209192290CE010E00E949B0A17C100912D
:105B80009129039500939129083018F007E00093BC
:105B90009129009191290E940C192091912902E1EB
:105BA00010E00E949B0A02C1E8E0F6E0008101FDDE
:105BB0001BC000E010E000936D2910936E29009344
:105BC0006B2910936C2904E610E00E94211406E072
:105BD0000E94620320E00EE010E00E949B0A20E099
:105BE0000FE010E00E949B0A00917229002309F542
:105BF00080916D2990916E29019680936D299093E3
:105C00006E29813008E0900734F000E018E000933E
:105C10006D2910936E2930916E29232F00E110E039
:105C20000E949B0A20916D2901E110E00E949B0ACD
:105C300020C080916B2990916C29019680936B29EB
:105C400090936C29883601E0900734F000E010E072
:105C500000936B2910936C2930916C29232F0EE04F
:105C600010E00E949B0A20916B290FE010E00E9437
:105C70009B0A20916D2930916E2900916B2910911A
:105C80006C290E94711202E00E9462038FC0009191
:105C90008229039500938229093018F008E00093C7
:105CA00082292091822904E110E00E949B0A7EC093
:105CB0008091692990916A2901968093692990932E
:105CC0006A29883601E0900734F000E010E0009384
:105CD000692910936A290091692910916A290E9403
:105CE000651130916A29232F07E010E00E949B0A7A
:105CF0002091692908E010E00E949B0A57C000919A
:105D00008C29039500938C29093018F008E0009342
:105D10008C2920918C2906EF11E00E949B0A46C035
:105D200000918F29039500938F29053018F004E026
:105D300000938F2920918F2907EF11E00E949B0A81
:105D400035C000919629039500939629093018F0E3
:105D500008E0009396292091962903EF11E00E9414
:105D60009B0A24C000919429039500939429043040
:105D700018F003E000939429009191290E940C19D6
:105D80002091942903E110E00E949B0A0E9445188B
:105D90000DC000918829039500938829003118F0DF
:105DA00000E00093882901E00093752908E210E0E3
:105DB0000E94211401E0009373290FC2E8E0F6E08D
:105DC000008101FD0AC200E00093400900917B2997
:105DD000E4EEF3E00C94A334E8E0F6E0008101FD8A
:105DE0002AC000E61AEE0E941C11B3950B2FB02FAB
:105DF0002091DA283091DB2810E02017310760F776
:105E000000918E29039500938E29053018F001E04A
:105E100000938E2920918E290DE010E00E949B0AAC
:105E200001E00093762900E510E00E94211403E0D0
:105E30000E946203D5C100917629002381F400916C
:105E400084290395009384290A3018F000E0009318
:105E500084292091842904E010E00E949B0AB6C1A5
:105E60000091A7290A950093A7290F3F19F400E094
:105E70000093A7290E941A192091A7290AEF11E07F
:105E80000E949B0AA3C1009187290A950093872944
:105E9000002319F40CE300938729209187290CEF44
:105EA00011E00E949B0A00E41CE90E941C118EC1B3
:105EB00000918D290A9500938D290F3F19F400E078
:105EC00000938D2920918D290DEF11E00E949B0AEE
:105ED00080918D2990E0019680932A0890932B0859
:105EE00075C18091C2289091C32801968093C228E1
:105EF0009093C328883E03E0900734F007EE13E048
:105F00000093C2281093C3280091C2281091C3287F
:105F100000932609109327090E9445183091C32841
:105F2000232F01E010E00E949B0A2091C22802E08A
:105F300010E00E949B0A4AC18091672990916829CC
:105F400001978093672990936829992332F408E692
:105F500011E000936729109368290E94961500911B
:105F60006729109168290093692910936A29309153
:105F70006829232F05E010E00E949B0A20916729E1
:105F800006E010E00E949B0A21C1009192290A9527
:105F9000009392290F3F19F400E000939229409159
:105FA000922950E00FEF10E00E94BD310E940A12CA
:105FB000209192290CE010E00E949B0A07C10091F9
:105FC00091290A9500939129013018F401E000937A
:105FD0009129009191290E940C192091912902E1A7
:105FE00010E00E949B0AF2C0E8E0F6E0008102FDAA
:105FF00011C000E010E000936D2910936E2900930A
:106000006B2910936C2904E610E00E94211406E02D
:106010000E946203009172290023F9F480916D2996
:1060200090916E29019780936D2990936E29992301
:1060300032F400E010E000936D2910936E29309146
:106040006E29232F00E110E00E949B0A20916D2908
:1060500001E110E00E949B0A1EC080916B29909183
:106060006C29019780936B2990936C29992332F4C2
:1060700007E611E000936B2910936C2930916C298D
:10608000232F0EE010E00E949B0A20916B290FE065
:1060900010E00E949B0A20916D2930916E29009199
:1060A0006B2910916C290E94711202E00E94620318
:1060B0008DC0009182290A95009382290F3F19F41F
:1060C00000E0009382292091822904E110E00E94DF
:1060D0009B0A7CC08091692990916A2901978093DD
:1060E000692990936A29892B31F408E611E000931D
:1060F000692910936A290091692910916A290E94DF
:10610000651130916A29232F07E010E00E949B0A55
:106110002091692908E010E00E949B0A57C0009175
:106120008C290A9500938C290F3F19F400E0009305
:106130008C2920918C2906EF11E00E949B0A46C011
:1061400000918F290A9500938F29013018F401E0FE
:1061500000938F2920918F2907EF11E00E949B0A5D
:1061600035C0009196290A95009396290F3F19F49E
:1061700000E0009396292091962903EF11E00E94F8
:106180009B0A24C0009194290A9500939429013018
:1061900018F401E000939429009191290E940C19B0
:1061A0002091942903E110E00E949B0A0E94451867
:1061B0000DC0009188290A95009388290F3F19F492
:1061C0000FE00093882901E00093752908E210E0B0
:1061D0000E94211401E00093732900E000937629C6
:1061E00000918629002311F40C94811D009164060E
:1061F0000F73009364060AE2009366290C94891DCC
:1062000000008895FECF0E94F034C801D9012A0110
:106210003B015CD057D071F48201930153D051F40B
:1062200001E2EEEAF9E2008341830FEF1FEF2FE76F
:106230003FE73DC044D0A201B3010E941733AC0137
:10624000BD0140D061F442D03AD00E9492340BEDAF
:106250001FE029EC10F43FE32AC03FEB28C0A20165
:10626000B3012DD00E94F133080119012FD0820112
:1062700093010E947A3423D0A0F41CD050F424D08F
:10628000A801B9010BED1FE029E430E40E945B3363
:106290000EC01AD04BED5FE069E470EC0E9417333A
:1062A00006C008D010F410D002C00ED03058E8E07C
:1062B0000C9401350E9492348001910108958C0163
:1062C0009D0108950C9470340C94F23740E050E036
:1062D00060E070E008953F7741E00C94913803E26C
:1062E0000DBF01E20EBFC0E0D1E20E949135002354
:1062F00011F00E9474380E9460190E9400310C94C1
:1063000000310D01DA0140E050E060E070E00E94F1
:10631000703439F400E010E04D934C9320E030E00D
:106320000CC0B901660F771F7E57572F550F550BBD
:106330007D935C932F7730783F63D00108950024DC
:10634000E8E0EA9532F0001F001C0416D0F3041AAE
:10635000F8CF001F402D00950895FF27442312F425
:10636000F1604195002312F4F09501950E949F3150
:10637000F0FD0195F1FD41950895149F102D059FA5
:10638000100D049F002D110D08954A951AF0000F6D
:10639000111FFBCF08954A951AF016950795FBCF6C
:1063A00008954A951AF015950795FBCF0895002496
:1063B0001124EFE0001F111F001C111C041615060C
:1063C00010F0041A150AEA95AAF7001F111FA00180
:1063D0000095109508955195419550400895FF27D7
:1063E000552312F4F160F7DF112312F4F09507D072
:1063F0000E94D731F0FD03D0F1FDEDCF0895119546
:106400000195104008952224349F302D259F300D92
:10641000169F300D079F300D249F202D310D159FA5
:10642000200D311D069F200D311D149F102D210DB3
:10643000321D059F100D211D321D049F002D110DD1
:10644000221D321D08954A952AF0369527951795F5
:106450000795F9CF08954A952AF035952795179510
:106460000795F9CF0895002411241001E0E2EA9580
:1064700092F0001F111F221F331F001C111C221C31
:10648000331C041615062606370688F3041A150A67
:10649000260A370AECCF001F111F221F331FA0014D
:1064A000B10100951095209530950895FF27772329
:1064B00012F4F16015D0332312F4F09509D00E9444
:1064C0003332F69508F404D0F69508F409C008951F
:1064D00030952095109501951F4F2F4F3F4F0895F0
:1064E00070956095509541955F4F6F4F7F4F089520
:1064F000FF27112477FB660F771F089409F4771F95
:10650000679517F8EE27002437FB220F331F0894F6
:1065100009F4331F279507F8089527FD0EC0EE0FE5
:10652000001F111F221F3A953230B8F7332319F498
:1065300027FD31E002C027FF30E0E03821F400FF02
:1065400008940EF488940F4F1F4F2F4F3F4F323057
:1065500038F4332319F427FD31E002C027FF30E07F
:106560003F3F29F0220F000C379527950895ACC0C6
:10657000032E002012F40E946832E02F012F122F08
:10658000232F3EE9D1CF0024F8CFBCDF432F4F5754
:1065900048F04F3148F007FC91C03FE72FEF1FEF65
:1065A0000FEF089533278CC0322F212F102F0E2F7D
:1065B0004F5141950E94233207FE08950C94683292
:1065C000F901EE0FFF1F37FBFF3F31F0EF2BE12BFF
:1065D000E02B8894B8940895E02BE12B21F00894E7
:1065E0009894B89408959894889438940895FB01E9
:1065F000EE0FFF1F77FBFF3F31F0EF2BE52BE42B76
:106600008894B8940895E42BE52B69F3E8CFEFDF85
:1066100068F021F43723262F8A010895372FFBCF06
:10662000E6DF20F00BF008957327EAF751C0C8DFCA
:10663000E8F3B3F361F3DBDFC8F383F3A1F358DFCF
:10664000401751076207730731F4011411F1002458
:10665000E89488942BC078F0332E372F732D322E88
:10666000262F632D312E152F532D302E042F432D21
:10667000302C012C132C371739F066955795479518
:10668000F795E0407395F7CFE7FBEE0FE0E01024BD
:106690006AF0EF0F041F151F261F60F4279517954A
:1066A0000795E79508F4689433953ECFEF0B040BFC
:1066B000150B260B39CFE0E87E27B9CF302D307887
:1066C00022271127002708953FE7302920E8F9CF36
:1066D0003FEF2FEFF6CF8BDFD8F3D1F3707837276A
:1066E000089585DFA8F3A3F3F9CF3078372793CF48
:1066F00067DF70F383F3A9F37ADF50F3B3F3A9F301
:10670000F7DE0124E8943F57E040370FEF1F12F007
:10671000D9F603C03A3E90F26894E0E00A92AA9358
:106720003A93AA27332422243327049FF001059F9C
:10673000F00D712D731F149FF00D711D221C069F0B
:10674000700D211C331C159F700D211C331E249FBE
:10675000700D211C331E169F200C311CAA1F259F73
:10676000200C311CA31F269F300CA11D39915EF413
:106770003395A695379427947795F795E7953395B4
:106780003130BCF316C0AA2322F0332351F43395E1
:1067900010C0339571F4A991099096CFA7FD09C057
:1067A0003A95EE0FFF1F771F221C331CAA1F3230B1
:1067B000A8F7E894FE2B09F068942A2F8101E72FAF
:1067C000A9910990BACE13DF10F00BF087CF80CFDC
:1067D0000EDFE9F3E0F3032E072670CF032E072622
:1067E00073CFEEDEA0F37BF399F301DF80F39BF32D
:1067F000A9F37EDE012427FD06C0000F111F221F12
:106800003150E040F8CF67FD06C0440F551F661FAA
:106810007150F040F8CFE894371BEF0B3158EF4F31
:106820002AF0EE23E9F63F3FD9F203C03A3EA8F240
:106830006894E0E0F0E011241394401751076207D8
:1068400038F0315008F46894000F111F221FEE1F1A
:10685000041B150B260BEF0B000F111F221FEE1F41
:106860000A9279E17A95AAF0041715072607EF072F
:1068700030F0041B150B260BEF0B089401C0889415
:10688000111C221C331C001C000F111F221FEE1FA5
:10689000E9CFF0F9E894E22BE12BE02B09F06894C2
:1068A0000694379427941794E79508F468947395A1
:1068B000B9F30990332311F0F0FF09C036942794FF
:1068C0001794E79508F4689433953130BCF3012DA3
:1068D000122D232D32CE8BCE9894089518940895BE
:1068E0006FDED0F3C1F383DEB8F304171507260774
:1068F000370708957CDEA0F063DE90F029F0E32FE7
:10690000E7273AF47317089572DE51F04EF00894B9
:106910000895041715072607370719F016F4B8F776
:106920008894089564DEE0F34BDED0F3E7DFC0F334
:10693000089408957591659155914591159011FAB6
:10694000259035900895F9DF041B10E003C0F4DFB3
:10695000041B150B20E030E005C0ECDF041B150B19
:10696000260B370BB8F010FC17C045910590E00FCF
:10697000F11F0417100540E02407340758F436F4DB
:1069800004910024F101E01BF0090994E00FF11FCC
:1069900025903590F101099411F4D6F7F1CF319695
:1069A0000EF0319650E060E070E045914B3F48F0CA
:1069B00089F34F3F29F04E3F11F075916591559144
:1069C0004591041B150B260B370B39F318F3E7CF52
:1069D000FA92EA92DA92CA92BA92AA929A928A9217
:1069E0007A926A925A924A92BA93AA939A938A9303
:1069F0000895FF84EE84DD84CC84BB84AA849984CA
:106A000088847F806E805D804C80BB81AA81998163
:106A10008881F0E0EC0FFD1FEF0108950E94EC3437
:106A2000229741E050E060E070E00E947A3460F428
:106A300040E00E94703421F402E26BD03FEF5FC06F
:106A400001E267D03FE75BC0AE010E948131C8011F
:106A5000D90143EF54E065E37FE30E947A3468F4A0
:106A600037FBAA0FBB1FB395B695A795B7F9088159
:106A70001981015010400883198340E050E060E81C
:106A80007FEB43D02801390140E050E060E87FE32C
:106A90003CD0A801B901820193010E94F133C801E1
:106AA000D901A801B9012FD0280139010881102F7F
:106AB000110F110B212F312F0E94B83248E152E7FC
:106AC00061E37FE320D04801590142E252E964EDDD
:106AD0007EE38201930117D04DED5BE96AE27FE32B
:106AE00016D0A201B3010FD044E050E060E070E4A2
:106AF0000ED0AC01BD0107D0A401B50108D022968B
:106B0000ECE00C94FD340C9478338C019D010C94D2
:106B10001733EEEAF9E2008351830FEF1FEF2FE7FF
:106B2000089501E008950E94E834EF97EF976A977F
:106B30002A873B874887598768017B0100E00B83E0
:106B40000C8302C011D21BD20AD2053251F00023AD
:106B5000C9F70B811C81EF96EF966A96E0E10C94E1
:106B6000F9340081053221F402D2FED105E2EBCFE7
:106B700000E00F830E830A8309833E0102E1600E69
:106B800000E0701E06E415E2088B198B06C009812F
:106B9000002311F400810983EAD1D9D10052B9F35D
:106BA000035059F00850B1F3025019F0035049F066
:106BB0000CC00A8103950A83EFCF0E8103950E83E3
:106BC000EBCF0F8103950F83E7CF00810A3279F471
:106BD000AAD1AD90BD9098D1BB203AF4B194A194C4
:106BE00000E0B00A0A8103950A83C1D114C0AA2427
:106BF000BB244AE050E00DC021916F0185010E9445
:106C0000BD31A22EBB24A00EB11E00EDA00E0FEFD1
:106C1000B01EA0D188F30A81002311F000E00F8399
:106C200096D10E32F1F4A3D192D10A3231F47BD154
:106C30008D909D9069D19BD117C0882499244AE0FA
:106C400050E088D188F421916F0184010E94BD3108
:106C5000822E9924800E911E00ED800E0FEF901E63
:106C6000F0CF88248A94982C80E071D10C5421F0C4
:106C70000C5131F0045039F481E0C80E7AD103C0D0
:106C800001E0C00ED81E6BD1EAE0F4E00C94A3340E
:106C900080FB5EF44B815C81652F660F660B47D1EC
:106CA00040835183628363834FCF2B813C813FD1EB
:106CB0002083318349CF37D10D91119625D10A8B8D
:106CC0002E0103E115D1E0C02ED16D907D901CD135
:106CD000062D072921F407E5602E05E2702E992084
:106CE00022F400E1802E07E2902E80E090E001C0C7
:106CF0000196F30101913F01002319F088159905D0
:106D0000BCF30CD12301919581959040680E791EBA
:106D1000BBC00E81002331F0082D092919F49924F4
:106D20008824839406E615E2088B198B08810037C6
:106D300039F4F9D0ECD000E1D5D000E0098330C0BF
:106D4000F1D046F40D911D912D913D91DDD0C801FA
:106D5000D90101C0DCD008810F3611F408E0ECCF76
:106D6000053749F70AE0E8CFDDD04D915D9126F473
:106D70006D917D91C9D005C0C7D0652F660F660B98
:106D8000762FCA01DB0177234AF40DE2098390953F
:106D9000A095B09581959F4FAF4FBF4F0AE0A2D00D
:106DA0003E0107E9600E00E0701E2E0107E9A0D049
:106DB000082F092B0A2B0B2B11F001E001C000E07A
:106DC0000D83082D092919F40D8100FF1FC094D0EF
:106DD000E889F989E00DF11D0081F30102933F017B
:106DE0008BD0C801D901012B022B032B81F79920ED
:106DF0006AF40F81002351F0A3D010E04501801AFE
:106E0000910A04C000E3F30102933F018E01095689
:106E10001F4F0619170908151905A4F30E81002341
:106E200099F10D8100FF30C00881083711F0083555
:106E300049F474D0F3010881008370D000E3F301BA
:106E4000008322C00F3601F5F30100810033E1F029
:106E500000E302933F0118C007E7602E05E2702EA1
:106E6000462C502EF2010081002371F001E040D049
:106E7000F9CF0FEFC00ED01E0AE9602E05E2702E8A
:106E80000DE9402E05E2502E420186189708A814FD
:106E9000B9041CF480E090E007C052D0A818B908EB
:106EA00010E0A01AB10AC5010A81002321F401C033
:106EB00063D00197EAF70981002339F055D004C067
:106EC00053D0F30101913F015AD00FEF800E901E75
:106ED000BAF70A81002309F437CE01970AF434CEB9
:106EE0004BD0FBCF10E00C871D871E871F870895AE
:106EF000400E00E0501E08954C855D856E857F85AF
:106F00008C019D010C943332A083B18308958D913F
:106F10009D91A083B183A0E0B0E008950FEF600ED3
:106F2000701E089580FBF701A081B1810895F701DB
:106F3000A081B1810D911D91A083B183F8010895C5
:106F40000981002311F001E0089500E00895F601A1
:106F500000810895F601008100530A300895F6017A
:106F600001916F010883089528853985089501E00E
:106F7000C00E00E0D01E08952885398500E2EA851C
:106F8000FB8509950B811C810F5F1F4F0B831C83B1
:106F900008950E94F434C801D9011A013F7740E8EE
:106FA00056E968E17BE40E94923438F416D0B3834A
:106FB00000E010E020E030E00DC03B2F0E94C53221
:106FC0000E94B8320AD03383A801B9018C019D0117
:106FD0000E945B33E4E00C940535F10100831183DA
:106FE000228308950E94E834C801D901BF7741E0A7
:106FF00050E060E87FE33B2F0E947A3470F440E079
:107000000E94703429F40BED1FE029E43FE350C0E7
:10701000CC24DD24EE24FF241CC00BEDC02E0FE099
:10702000D02E09E4E02EF72E40E07FEB082F48D069
:107030002801390140E050E060E87FE38C019D01C8
:107040003FD0A801B901820193010E94F133C80128
:10705000D901AC01BD018C019D012DD02801390160
:1070600044E25FEF6BE27CEB26D048E854E466EA4A
:107070007EE328D048E150EC6FE370E423D045EB89
:107080001CD0480159014AEE54EB66E870E48201D5
:10709000930118D046EB11D0A801B90184019501E4
:1070A0000E94F133AC01BD0106D0A601B70108D0A2
:1070B000E0E10C94F9340C9478335DEF68E670E409
:1070C0000C941733FDDFA201B301F5CF20E006D009
:1070D000E9F70895259102D0E9F708952D9301501D
:1070E0001040202F212B089582EA93E7FC0105919F
:1070F0001491FC013296A591B491FC01349625912E
:107100003491422F432B19F0F901E4DF01C0DEDF97
:10711000069613E78E3A910748F3089540E00C94E1
:1071200091380E94F0342897802FB32F442E40E0EE
:1071300050E060E070E00E947A3410F401E001C099
:1071400000E0000F400EBF7743E859EF62E27FE3B3
:10715000082F3B2F80D076D041E05CEF6FE777E4DB
:107160000E94923488F5AE010E94C9376BD0042D7D
:1071700010E06BD0488159816A817B8172D008838D
:1071800019832A833B83AE014C5F5F4F2A0140E0A5
:1071900050E060E87EE35FD0A2010E94C93740E082
:1071A00050E060E870E40C811D812E813F8153D056
:1071B000A801B901088119812A813B810E945B33B2
:1071C0000E94C532402E0CC00E94C532602E3DD0B8
:1071D000A801B9018C019D0133D0460C03E0402287
:1071E00040FA3EF4AC01BD0100E010E020E83FE3CE
:1071F00027D002E0401608F0B0588C019D0129D03C
:10720000280139014BEF57ED6EE179E324D045E6D3
:1072100056E269E97BEB21D048E554E363EA7DE37C
:107220001CD041EE5DE565E27FEB17D04BED5FE0F2
:1072300069EC7FE316D00DD02896E8E00C94013578
:107240000E945B33C801D901089520E030E00C941E
:10725000C332AC01BD010C94783303D0A201B30159
:10726000FACF0C9417331B2F6A2FF901A081B1813B
:10727000AD014F5F5F4F408351830C93A62FB12F19
:107280000895BA93AA9324970A831B8389019E01C8
:107290002A5F3F4F28833983BE01AE014E5F5F4FA7
:1072A00023E339E30E94933520E0AA81BB812C932C
:1072B0002496A991B99108950E94EC34229748012F
:1072C000590141E050E060E070E00E947A3498F4A7
:1072D00040E00E94703429F400E010E020E030E04B
:1072E0004EC001E2EEEAF9E2008351830FEF1FEF97
:1072F0002FE73FE744C0AE010E948131C801D901A8
:1073000045EC53E062E47FE30E9417334AE151E524
:1073100062E17FE33BD0A801B9018C019D013BD024
:10732000402E088100FF14C00A952DD0802F43EF16
:1073300054E065EB7FE3042D0E94783337FB220F86
:10734000331F380F3695279537F9C801D9010BC07F
:107350001AD0842D912FD90137FBAA0FBB1FB00F74
:10736000B695A795B7F940E050E060E87EE38C0160
:107370009D010CD0AC01BD01840195010CD0229679
:10738000ECE00C94FD3442E00C94AD310E94783373
:107390002801390108950E94F133A201B3010C9430
:1073A00017337A042421AE7312049E2500004E6F19
:1073B000726D6100547572626F005472657368007B
:1073C0004F6666004F6E004F6E2B004F6C6400449A
:1073D000796E00442B53007664692000564449209E
:1073E00000537664690053564449002D20504C45A3
:1073F0004153452057414954202D20002020202072
:107400002020203C3E2020202020202000204C6FE7
:107410007720426174746572792021212100204512
:10742000524153494E4720454550524F4D2120006F
:10743000202A726164696F646F6D2E6F72672A20F3
:10744000004B504F54322D4741494E2D533620208A
:107450002563200050726F663D25642000466163FD
:10746000746F72792073657474696E67730020207D
:107470002053657474696E677320202020200055A6
:107480003D256420493D256420456D3D256420202F
:1074900020004D3D256420413D25642047623D2567
:1074A000642025642A256420005458202564487AE5
:1074B0002025646D4120200052582025646D5620FF
:1074C0002020200025642A25645F257320002020C9
:1074D000205475726E20636F696C21003C20256416
:1074E000206D56203E00436F696C20626C3F20592E
:1074F000657320272B2700202020202020202020FB
:1075000000202564256446256425630025647625CE
:107510006420002B253032645B002D253032645B03
:10752000005D205325642564462564256300256499
:107530007625640020202020202F202020202020BD
:1075400020202020002020202020202050502020FB
:1075500020202020200025642020202020200050F2
:10756000726F66696C65202020202020202020007A
:1075700054623D25642E256456202055623D2564C5
:107580002E25645620004261747465727920202093
:1075900020203C25643E002B2564202020202D2E19
:1075A0002E2E2E2E2E2E2E2B00436F6E74722E201A
:1075B000202020202020202020200025646D412034
:1075C00020202020202020202020202020002825CE
:1075D00064292E2E2E20002A467265715F54582091
:1075E000256C64487A20002A4665727269746520A9
:1075F000200020202564256320200025646D412083
:1076000020200025632D2E2E2E2E2E2E2E2B0050C8
:107610006F7765722E20202020202020202020003F
:107620002A2564202A256420002D2E2E2E2E2E2E73
:107630002E2E2B004761696E202020202020202044
:10764000202020200025646D5620202020202000AE
:1076500020413D2564202020002A436F696C206270
:107660006C2E20663D2564256320200025642020A3
:1076700020202000485046202020202020202020AC
:10768000202020200047726F756E6420626C2E20CF
:1076900000534C2E25732000566F6C756D652020AD
:1076A0002020202020202020002564746F6E65207B
:1076B000200025732D2E2E2E2E2B00426565707313
:1076C0002020202020202020202020002573256439
:1076D000202D2E2E2E2E2E2E2E2E2B00496E642B7C
:1076E00041752020202020202020202000257320EC
:1076F0002D2E2E2E2E2E2E2E2E2B004D6F6465201D
:107700002020202020202020202020200038363457
:1077100032302F30313233343536373853004772F8
:107720006F756E6420626C2E4572726F7221004715
:10773000726F756E6420626C2E202D4F4B2D2000D1
:107740002020202A2A2A202564202A2A2A202020B4
:1077500020002020202825303264293C2530326446
:107760003E2020202020002020202020202020201B
:10777000202020202020200020204E6F20466572EF
:107780007269746521202020002054616B652046B9
:107790006572726974652120200020202020204518
:1077A00072726F72212020202020002020202020B3
:1077B000204F4B212020202020202000202020208E
:1077C00020206C6F6E672020202020202000900158
:1077D0003031323334353637383941424344454607
:1077E00000286E756C6C20706F696E74657229006C
:1077F0003031323334353637383961626364656627
:1078000000464C4F4154533F2077726F6E6720669D
:107810006F726D617474657220696E7374616C6CE3
:08782000656421003F3F3F00B9
:0400000300000000F9
:00000001FF
